:100000004FC3000085C3000083C3000081C300000C
:100010007FC300007DC300007BC3000079C30000E4
:1000200077C3000075C300000C94D5310C94BD3229
:100030000C948A316DC300006BC3000069C30000DB
:1000400067C3000065C3000063C3000061C3000014
:100050005FC300000C94B1315BC3000059C30000C2
:1000600057C3000055C3000053C3000051C3000034
:100070004FC300004DC300004BC3000049C3000044
:1000800047C3000045C3000043C3000041C3000054
:100090003FC300003DC300003BC3000039C3000064
:1000A00037C3000035C3000033C3000005010980D9
:1000B000A101850319012AB700150126B700950192
:1000C00075108100C0050C0901A101850419012AE0
:1000D000A002150126A002950175108100C005013E
:1000E0000906A1018506050719E029E71500250184
:1000F0009508750181020507190029EF15002501F2
:1001000095F075018102050819012905950575010C
:100110009102950175039101C00660FF0961A1017B
:100120000962150026FF00952075088102096315F4
:100130000026FF00952075089102C005010906A15F
:1001400001050719E029E7150025019508750181CA
:10015000029501750881010507190029FF15002680
:10016000FF0095067508810005081901290515008D
:100170002501950575019102950175039101C00056
:10018000000000000000000000000000000000006F
:10019000000000000000000000000000000000005F
:1001A0000000007E0F00D4FFFFFFC70000007800B2
:1001B000000000000000002A2B28000000000000C2
:1001C0000000000000000000000029000000002CDA
:1001D0001E3420212224342627252E362D37382779
:1001E0001E1F202122232425263333362E37381F85
:1001F0000405060708090A0B0C0D0E0F1011121347
:100200001415161718191A1B1C1D2F3130232D35E4
:100210000405060708090A0B0C0D0E0F1011121326
:100220001415161718191A1B1C1D2F3130354C09BF
:10023000025B00030100A0FA0904000001030101B0
:100240000009211101000122440007058103080073
:10025000010904010002030000000921110100014D
:100260002222000705820320000107050303200066
:10027000010904020001030000000921110100012D
:10028000226D000705840320000112010002000016
:10029000000869EB01650100010203011C037600FF
:1002A000690061006C003A006600360034006300AB
:1002B000320062003300630000001203410070004E
:1002C0006500720074007500720065000000100384
:1002D000420069007A0075006E006F007700000030
:1002E0000403090429001E001F0020002100220031
:1002F000230024002500260027002D002E003100B9
:100300004A002B0014001A000800150017001C00FA
:1003100018000C00120013002F0030002A004B00C0
:10032000390004001600070009000A000B000D0048
:100330000E000F003300340028004C004E00E10096
:100340001D001B00060019000500110010003600FA
:10035000370038000000E50052002152E000E300C1
:10036000E2000000000000002C000000000000007F
:10037000E6000000500051004F0001003A003B0031
:100380003C003D003E003F00400041004200430071
:1003900044004500010001000100010001000100CE
:1003A0000100010001000100010001000100010045
:1003B0000100010001000100010001000100010035
:1003C0000100010001000100010001000100010025
:1003D0000100010001000100010001000100010015
:1003E0000100010001000100010000000100010006
:1003F00001000100010001000000000000000100F8
:1004000000000000000001000000010001000100E8
:1004100001000100B604CA151E1600000200020009
:10042000B204CA151E16000003000100B704CA1565
:100430001E160000040002009C04CA151E16BE070A
:1004400005000100B804CA151E16000006000200CF
:100450009E04CA151E16000007000200B404CA1547
:100460001E16000012000200BA04CA151E16000073
:1004700013000200BC04CA151E160000140001007F
:10048000BE04CA151E160000150000000000C707B4
:10049000670E000016000100B904E11535160000D2
:1004A00017000101B904E11535160000180001021A
:1004B000B904E1153516000019000200C004CA1580
:1004C0001E1600001A000103B904E11535160000DC
:1004D0001B000200C204CA151E160000FD377A5820
:1004E0005A000004E6D6B4460200210116000000BE
:1004F000742FE5A3E002B1010D5D003D8889C6546B
:1005000036C3174FE4DB9EFB41790B8A1053BDFFC6
:10051000AE6112D5352534C52305731BC3909EB13A
:10052000A3FEBD5FE0D8E3F08C143450FFB57CA788
:10053000D26CC36177D4B8A9FB8F54967383FEBE87
:100540002816E5D7A78B99AAB3E997AB282EE5E73C
:10055000B479CE2A676F28FCAE9157BD88C5541F69
:100560000106D235B4408D2F17FB786FC1A42D53EF
:1005700049B50DA015CAF6F2269A863562FD46FAEF
:1005800085F499ABFE6E899B31763C42FAB6745283
:10059000DC87631C6D5C87AFE40D97D47E1569F42E
:1005A000C39AE29AA0C3DD51399171B4B654FA935B
:1005B000CA53BDC6E67C7F939B13E445612BA8AD6F
:1005C0006A5D6A2F1917F51E4499281BCECE95F146
:1005D000E95CA5295707AFD98CB503E04DB7C3C572
:1005E00037AC8FE511BA4C675A2D8D1FD3655BFB75
:1005F0003ADB7118155E1488381AD5F532D0B65921
:10060000FE3B7FEF893E7E00000000009B4F48BC10
:100610008B3592E60001A902B205000061833636EF
:10062000B1C467FB020000000004595A4C4C4C4C0A
:100630004C4C4C52525252525252524C4C4C4C4CCA
:100640004C4C52525252525252524C4C4C4C4C4CBA
:100650004C52525252525252524C4C4C4C4C4C4CAA
:1006600052525252005252524C4C4C0000002A003E
:1006700000005200525252504F52514A4D4B4E2A96
:100680004C2F30B6B7ABACBBBCA9AABDBE0D0E0B90
:100690000F1A0508050905071811130408120C00A4
:1006A00011241FBECFEFDAE0DEBFCDBF04B603FEDC
:1006B00018C08091C9049091CA04A091CB04B09154
:1006C000CC048730904BA740B04B59F41092C9042A
:1006D0001092CA041092CB041092CC04E0E0F8E32C
:1006E000099511E0A0E0B1E0E0E4F8E602C0059071
:1006F0000D92AE3AB107D9F724E0AEEAB1E001C0FD
:100700001D92A93CB207E1F70E94FA2A0C94E33348
:1007100077CC9C019A9581159F4118F5F32FF270C3
:10072000EE27832F8170732F74706627532F5870B4
:10073000442734FF0CC08295807FEF2B09F0806244
:10074000672B09F08064452B69F080680895EF2BD2
:1007500009F08260672B09F08460452B19F08860EE
:10076000089580E00895CF93DF93EB01D2DFFE017F
:100770000995DF91CF9108950C940E330895982F29
:1007800092959F7024E0911102C020E0982F892F4C
:1007900086958695811511F02E5F982F892F869565
:1007A000820F0895282F92959F70963099F060F4EB
:1007B000925F9F70923030F4203FB1F038F481E0C6
:1007C000283E38F080E008959A5FF3CF81E0243F1F
:1007D000C9F7089591E0813F09F090E081E0283E5B
:1007E00008F080E0892B089581E0089580933E040D
:1007F000089580933F04089521E030E001C0220F66
:100800008A95EAF780913F04822BF3CF21E030E014
:10081000A90102C0440F551F8A95E2F7CA018095CD
:1008200090913F048923E5CF292F953090F58F30A3
:1008300080F590E03FE0239F800D911D1124282F2B
:10084000277041E001C0440F2A95EAF723E096950E
:1008500087952A95E1F7FC01EE0FFF1FE80FF91FBE
:10086000ED56FD4F20E030E070E05191DF01CB010B
:10087000022E02C0969587950A94E2F781708195C1
:100880008527842385278E932F5F3F4F23303105A3
:1008900061F70895292F953078F58F3068F590E04D
:1008A0003FE0239F800D911D1124682F677023E086
:1008B000969587952A95E1F7FC01EE0FFF1FE80F4B
:1008C000F91FED56FD4F40E050E080E0219130E00F
:1008D000062E02C0369527950A94E2F72170332739
:1008E000042E01C0220F0A94EAF7822B4F5F5F4F5C
:1008F0004330510559F7089580E0089590913F04E1
:1009000021E030E0F90101C0EE0F8A95EAF7D90144
:1009100002C0AA0FBB1F6A95E2F7EA2B01C0220FA3
:100920004A95EAF7892F8E23E81303C0892F822B7B
:1009300060CF2095822F8923FBCF8091920290E097
:1009400020E0022E001C0008281709060CF008956C
:100950002F5FF7CFFC01DB018481813041F51496D4
:100960008C911497813019F591818FE0E081F0E04E
:10097000899FE00DF11D1124E45DF94F94919A32A5
:10098000B1F011962C911197EC91F0E0829FE00D5F
:10099000F11D1124E45DF94FE49181E09E1301C043
:1009A00080E091E0EA3209F090E0892B089581E03F
:1009B00008959C01809140048D79811119C0211501
:1009C00040E5340780F4211580E23807C0F4233372
:1009D000310511F1D0F481E02E31310590F424304D
:1009E000310530F00895C90196558115914010F0F8
:1009F00080E00895C901805F96450797C8F33327C3
:100A0000E6CF2C323105A1F708952653310981E054
:100A10002330310538F3ECCF81E0089580914A040A
:100A200090914904981301C008958F5F8770FACFA1
:100A3000909144048095892380934404282F277043
:100A4000211110C0891771F09091C50492FF0AC05E
:100A5000869586958695DADE1092440410924604B7
:100A600010924504089590914004982B909340046F
:100A70000895982F90958091400489238093400495
:100A80000895982F9095809143048923809343047F
:100A9000089580913C04811531F010923C0410922D
:100AA0003B0410923A040895803E9105D9F1C8F4B0
:100AB0008133910509F482C048F48932910509F423
:100AC00072C08A32910509F480C008958933910576
:100AD000E9F082389105D1F08533910509F45EC0C3
:100AE0000895843E9105D9F148F4823E910539F18B
:100AF000833E910549F181EE90E00895863E91058F
:100B0000C9F1873E910509F43EC008952091C404BF
:100B10002370211164C02091C50423FF14C089E211
:100B200090E008952091C40420FD45C03091C50493
:100B300030FF09C024FD24C083EE90E00895209189
:100B4000C40422FDF7CF08952091C40422FD44C0BF
:100B50003091C50430FD43C024FFF5CF11C0209172
:100B6000C50421FFF0CF8091C40484FD09C087EE45
:100B700090E008952091C40423FFE5CF24FFF7CF30
:100B800080E090E008952091C40423FD2BC03091B3
:100B9000C50431FFE1CF84EE90E008952091C404B4
:100BA00025FFD1CFBCCF2091C40425FD1EC02091CC
:100BB000C50423FFC8CF89E390E008952091C404C1
:100BC00026FFC1CF8AE290E008952091C40426FF59
:100BD000BACF81E390E0089582EE90E0089580EE30
:100BE00090E0089586EE90E0089585E390E0089502
:100BF0009091C40492FF10C041E0282F247124304A
:100C000009F040E031E0282F2871283009F030E069
:100C1000431711F02CE0822793FF10C041E0282FEA
:100C20002471243109F040E031E0282F2871283167
:100C300009F030E0431711F02CE082273091C50411
:100C400030FF10C051E0282F2171213009F050E011
:100C500041E0282F2871283009F040E0541711F0A6
:100C600029E0822731FF10C041E0282F2171213176
:100C700009F040E031E0282F2871283109F030E0F8
:100C8000431711F029E0822794FD877E08951F9372
:100C9000CF93DF9309DFEC01811522E5920708F07D
:100CA00052C0811540E5940708F0CDC0803E910503
:100CB00020F58D3C910508F0A1C0883A910570F4AB
:100CC000853A910508F097C081309105B9F10497F4
:100CD000813A910598F1C0E0D0E030C0885A91097E
:100CE0004B97C8F7C85AD0E0CC0FDD1FCF5BDE4F63
:100CF0000990D881C02DD46421C0811550E4950796
:100D0000B0F4C11580E2D80708F0B3C0C83ED105E1
:100D1000A8F0CE019A9581159F41E8F68D2F68DFE6
:100D2000182FCE019927C0DEEC01D12B07C09927DF
:100D3000BBDECC27DF70C82BD92BD06ACE01DF9168
:100D4000CF911F910895803842E59407C8F5803609
:100D500052E5950708F05BC0C03482E5D807D0F4AF
:100D6000C03292E5D90708F04BC08C2F8695869546
:100D700020E2829FC0011124C37021E030E0A9016C
:100D800002C0440F551FCA95E2F7EA01C82BD92BC0
:100D9000DD68D4CF8C2F86958695877050E2859F2D
:100DA000C0011124C37021E030E0A90102C0440F4A
:100DB000551FCA95E2F7EA01C82BD92BDC68BECFD4
:100DC000803C52E5950758F48F71C03AD245A0F5A2
:100DD00090E0982F8827EC01C46FD06AAFCF805C79
:100DE0009245809708F077CFDC2FCC27CC27DF7196
:100DF000C06FD06AA3CFA497D064A0CFD0659ECF98
:100E0000CF71D0E0DC2FCC27C16FD06A97CF869509
:100E10008695877020E2829FC0011124C37021E073
:100E200030E0A90102C0440F551FCA95E2F7EA015C
:100E3000C82BD92BDA6882CFDBDEC82FD0E0DC2FBD
:100E4000CC27D0627BCF8F71D3DE93E0CC0FDD1F38
:100E50009A95E1F7CC27DF70282F30E084FF05C09A
:100E600050E1859F900111243327C22BD32BD069E9
:100E700065CF8D2F8F71BCDE182FCE01992714DE20
:100E8000EC01D12BDECF80E00895F894E82FE295B5
:100E9000EF70F0E041A18F7021E030E0B90102C0B5
:100EA000660F771F8A95E2F7CB01962F90959423D2
:100EB00091A392A1892B82A37894089581152CE7A0
:100EC000920741F420914F0230915002232B11F4EC
:100ED00080E090E00895E6EAF3E080E090E062E1EF
:100EE0007AE245E35AE227EA3AE27783668351875A
:100EF0004087338722879787868701967096883048
:100F0000910599F70895FB01811520E2920728F4D5
:100F1000811541E0940738F408959C013052211561
:100F2000304348F00895392F94FF02C03295307F46
:100F30002081232B208399270895462B22FF0FC061
:100F4000982F92959F708F70892B962F92959F70F6
:100F50006F70692B942F92959F704F70492B982F2B
:100F60009623961309C050E04095509590E0482391
:100F7000592381E0452B09F080E0089580919C047D
:100F800090919D0490930D0180930C010895EF9230
:100F9000FF920F931F93CF93DF93FB018FEF9FEF90
:100FA0004430510508F45FC04091C40441FB8827D8
:100FB00080F990E0880F991F42FB002700F910E0AC
:100FC000000F111F000F111F802B912B40FBEE24EF
:100FD000E0F8F12C8E299F2943FB222720F9C22F0C
:100FE00050E0D52F53E0CC0FDD1F5A95E1F78C2B45
:100FF0009D2B44FB222720F950E1259F90011124CD
:10100000822B932B45FB222720F950E2259F90014C
:101010001124822B932B46FB222720F950E4259F95
:1010200090011124822B932B47FB222720F940E8C3
:10103000249F90011124822B932B2091C504322FE1
:101040003170932B26952170B22FBB0FA0E08A2B15
:101050009B2B092E000CAA0BBB0B80839183A283D0
:10106000B38380E090E0CDB7DEB7E6E00C944D337B
:10107000AC0123E0969587952A95E1F78E71992723
:10108000FC01E850FE4F0190F081E02D4F70552794
:1010900021E030E002C0220F331F4A95E2F76115CC
:1010A00041F0E22BF32B88509E4FDC01ED93FC9333
:1010B000089520953095E223F323F5CFFC01848138
:1010C000862381110AC082818115B9F06823908539
:1010D00093FF05C081E061110FC080E00895282FC3
:1010E00022952F708F70282B962F92959F706F707E
:1010F000962B81E02913F1CF089581E008950F9395
:101100001F93CF9301E010E0082E01C0000F0A9456
:10111000EAF7C09139049C2F9023911115C090914A
:101120004404969596959695891306C010924404AA
:1011300010924604109245045FDBC027C093390427
:10114000CF911F910F91089561DBF7CF9091080324
:1011500089029001112437FF03C08093080308958A
:101160002F3731051CF4980F9093080308959C01C4
:1011700080E090E0F901E80FF91FE491E41307C063
:1011800091E08927F901E80FF11D849108950196F6
:10119000861780F380E00895FA01309709F00995E9
:1011A0000895E0917802F0917902309739F001903A
:1011B000F081E02D309711F00995089580E00895B1
:1011C000A3E0B0E0E6EEF8E00C9435339C018091AA
:1011D000F6019091F70182179307B1F03093F70170
:1011E0002093F601E0917802F0917902309761F056
:1011F0000084F185E02D309739F083E089833B83CB
:101200002A83CE01019609952396E2E00C9451338E
:10121000A3E0B0E0EEE0F9E00C9435339C0180915E
:10122000F4019091F50182179307B1F03093F50125
:101230002093F401E0917802F0917902309761F007
:101240000084F185E02D309739F084E089833B8379
:101250002A83CE01019609952396E2E00C9451333E
:1012600090911001913091F0A2EBB1E0EFEF90E09E
:101270002D91821751F0EF3F19F4211101C0E92F90
:101280009F5F9630A9F7EF3FC9F408959091C40489
:1012900097FFEACFE82FE695E695E695803FA8F719
:1012A000F0E0E854FE4F877021E030E001C0220FEB
:1012B0008A95EAF78281822B828308950E2E000C94
:1012C000FF0BE055FE4FF8CF90911001913021F4C3
:1012D0009091C40497FD0CC0E2EBF1E09191891369
:1012E00002C0DF011E9251E0E83BF507B9F708950F
:1012F000E82FE695E695E695803FC8F7F0E0E854DC
:10130000FE4F877021E030E0A90102C0440F551F55
:101310008A95E2F7CA018095928189238283089594
:1013200080910F0108952FB7F8948091F00190916A
:10133000F101A091F201B091F3012FBF08958091C6
:101340009E0490919F04892B89F0EDDF20913A044F
:1013500030913B04AC01421B530B9A0181E0409158
:101360009E0450919F042417350708F480E00895E7
:10137000CF93DF93C091400480914304C82B8091A8
:101380003C048115E1F080919E0490919F04892B8B
:1013900019F0D5DF81117DDBD0913C0480911001E3
:1013A000813021F48091C40487FD13C086E022EBD4
:1013B00031E090E0815088F491116BDBCD2B80916E
:1013C000220380958C2390912103892BDF91CF916B
:1013D00008958EE12AEB31E0ECCFF90141919F01B4
:1013E000411541F39F5FE6CF962F2091C50422FF60
:1013F0000EC0682F660F660F660F692B609344045A
:10140000FBD991DF90934604809345040895F4C975
:1014100090913C04292F2823211559F08095892388
:1014200080933C04811531F07EDF80933A049093E1
:101430003B04089580E090E0F8CFCF93C82F8091CF
:10144000C50482FF0BC080913C048C1739F06BDF20
:1014500090933B0480933A04C0933C04CF91089549
:101460002FB7F8946091F0017091F1018091F20131
:101470009091F3012FBF0895CF92DF92EF92FF92E8
:10148000CF93DF93D82FC92FC090A003D090A10392
:10149000E090A203F090A303E3DF6C197D098E09AD
:1014A0009F09643F71408105910510F1D9DF6B01FF
:1014B0007C0182E390E0A0E0B0E0C0923C02D092D8
:1014C0003D02E0923E02F0923F02809338029093F8
:1014D0003902A0933A02B0933B02D0939E03C0938B
:1014E0009F03DF91CF91FF90EF90DF90CF90089511
:1014F00084EF91E0A0E0B0E0E0CF0895FC019B0113
:101500008091E6019091E7018617970740F0672BDD
:1015100029F48091E8008E778093E800C90140E0CB
:10152000009741F4411106C08091E80082FF2FC06E
:1015300080E00895209151022115A9F12530A9F1EB
:101540002091E80023FD2DC02091E80022FDECCF82
:101550002091E80020FFE4CF3091F3002091F200C9
:10156000009719F02830310558F041E02830310556
:1015700009F040E02091E8002E772093E800D0CFDA
:1015800041914093F10001972F5F3F4FE9CF809148
:101590005102811541F0853041F08091E80083FFD0
:1015A000C3CF81E0089582E0089583E0089580919B
:1015B000E00187FF13C08091E80082FF06C08091A0
:1015C000E8008B778093E8000895809151028111A3
:1015D000F2CF0895809151028115D9F38091E800EE
:1015E00080FFF8CF8091E8008E77ECCF2091E40067
:1015F0003091E50095E6A9012091EC00822F8170E1
:1016000020FF06C08091E80080FF06C080E00895BA
:101610002091E80022FD1AC080915102811589F0C5
:10162000853089F08091EB0085FD0FC02091E400AA
:101630003091E50042175307F9F29A95E1F684E0FC
:10164000089582E0089583E0089581E00895E8ED2B
:10165000F0E080818E7F80831092E2001092DA00A9
:101660001092E100A0EEB0E08C9181608C938081BB
:101670008F77808319BCA7EDB0E08C918E7F8C931F
:1016800080818F7E80831092DF010895E09178023F
:10169000F0917902309739F00284F385E02D30978C
:1016A00011F060E209950895982F9093E900891749
:1016B00071F07091EC002091ED005091F00021FD4F
:1016C00009C09F5F973089F78093E9000895762FCE
:1016D000242F50E03091EB003E7F3093EB003091AF
:1016E000ED003D7F3093ED003091EB0031603093A1
:1016F000EB007093EC002093ED005093F0002091EC
:10170000EE0027FDDECF0895A0E0B0E0EAE8FBE0C0
:101710000C942F33C8EDD0E088818F7E8883E7ED6D
:10172000F0E080818160808384E082BF81E08093EB
:10173000DF0188818E7F888302EE10E0F80110823D
:101740001092DA0081EEC82ED12CF6011082888129
:101750008F77888388818068888388818F7D88835C
:1017600019BC109251021092DE0110922C021092BC
:10177000DD0190EEE92EF12CF70180818B7F8083D3
:1017800088818160888342E060E080E08DDFF6013F
:1017900080818E7F8083F801808181608083808159
:1017A00088608083F70180818E7F8083888180615B
:1017B0008883CDB7DEB7E8E00C944B33E0914A0460
:1017C0009091490429E0E91302C080E00895AE2F0A
:1017D000B0E02E9FF0011124E55BFB4F3181361301
:1017E00006C03081381303C03581341304C0FD01B5
:1017F0003196E770E8CF81E008959C01211531050D
:1018000009F408958FE99FE00197F1F700C0000007
:1018100021503109F3CF81E08093E00080E2809392
:10182000D8001092C9008FE19EE40197F1F700C043
:10183000000087E090EBDC018093C9049093CA0418
:10184000A093CB04B093CC0488E19CE00FB6F8944D
:10185000A895809360000FBE90936000FFCF0F9318
:101860001F93CF93DF938B01EA0190915102943043
:1018700051F58093E9008FEF9091E80095FD06C047
:1018800095ED9A95F1F700008A95B1F78091E800FF
:1018900085FF19C0ABDE811111C08091E80085FD84
:1018A00006C08091E8008E778093E800F3CFF801BE
:1018B00081918F018093F100219779F78091E80061
:1018C0008E778093E800DF91CF911F910F9108955B
:1018D000792F603229F440E250E0682F82E0BFCFD8
:1018E0000895CF93DF93D82FC92F48E050E0682F99
:1018F000792F81E0B4DF88E0ED2FFC2FA8EEB1E076
:1019000001900D928A95E1F7DF91CF910895BC0186
:1019100040E250E084E0A3CFBC0143E050E084E02B
:101920009ECF9091C50492FB222720F9281771F0D1
:1019300080FB92F99093C5046091C4047091C50432
:1019400084E090E00E94C83382E072C808951F933B
:10195000CF93DF93962F122F632F8430D8F49530D6
:10196000C8F44F30B8F4C42FD0E0CC0FDD1F2EE107
:10197000929FC00DD11D112496E9899FC00DD11DE4
:101980001124CE0189960E94AE33612FCE018A9632
:101990000E94AE33DF91CF911F9108958091100185
:1019A000813061F58091C40487FF28C0E1DC809319
:1019B000B90140E250E068E572E088EB91E00E94F6
:1019C0006533892BD1F080E2E8EBF1E0A8E5B2E0E5
:1019D00001900D928A95E1F7E0917802F0917902F9
:1019E000309759F00480F581E02D309731F086E092
:1019F0008093B80188EB91E009950895B9DC809354
:101A0000B00148E050E06AE772E080EB91E00E94AC
:101A10006533892B91F388E0E0EBF1E0AAE7B2E0CF
:101A200001900D928A95E1F7E0917802F0917902A8
:101A3000309719F30280F381E02D3097F1F280EBBB
:101A400091E0DACF811511F00ED8A8CF0895811555
:101A500031F090914304892B809343049FCF0895E4
:101A6000811511F006D89ACF0895811511F009D883
:101A700095CF089580911D03811521F082E2F5DF55
:101A800010921D030895CF93C82F8115C1F08CEFDC
:101A90008C0F813A80F580911001813021F4809182
:101AA000C40487FD0EC0E2EBF1E08191C817F9F0A4
:101AB00021E0E83BF207C9F78C2FD2DB6FDFCF9133
:101AC0000895EC2FE695E695E695F0E0E854FE4F94
:101AD000828190E04C2F477021E030E002C0220F5D
:101AE000331F4A95E2F782239323892B29F38C2F06
:101AF000EBDB54DFE1CF80E28C0F883048F4C77015
:101B000081E001C0880FCA95EAF70E943305D6CF5D
:101B10008BE58C0F833030F42C2F2452330BC9010A
:101B20004FDBCDCFC85ACB3150F6EC2FF0E0EE0FA3
:101B3000FF1FE958FE4F808191816ADBC0CFCF93B0
:101B4000DF93EC01805E9109089720F067E27DE069
:101B5000209711F462E27DE0CE010E94B3038C2F46
:101B600092DFDF91CF910895611529F02091430410
:101B70002260209343049C0130522115304308F425
:101B80009927DDCF811509F19CEF980F913A10F458
:101B90009BDB04CF90E2980F983050F4877091E06F
:101BA00001C0990F8A95EAF7892F0E943905F1CF74
:101BB0009BE5980F933018F480E090E001CB885AB1
:101BC0008B3118F480E090E023CB0895CF93DF931E
:101BD000EC01D8DFCE01805E9109089720F065E323
:101BE0007DE0209711F460E37DE0CE010E94B30315
:101BF000DF91CF9108951F93CF93DF93182FEB01BF
:101C000042DF209731F4812FBDDFDF91CF911F910B
:101C100008958FE99FE00197F1F700C00000219738
:101C2000F0CF6091BC047091BD04893321F06091C4
:101C3000BA047091BB04DFCF109240048091100170
:101C40008130A1F48091C40487FF10C0EAEBF1E079
:101C50008EE1DF011D928A95E9F780E090E0B0DA2D
:101C600080E090E0D5DA1092430498CEE2EBF1E008
:101C700086E0EFCFE1DF2FEF84E39CE0215080404E
:101C80009040E1F700C0000088E19CE00FB6F894B6
:101C9000A895809360000FBE90936000FFCFCF9314
:101CA000DF93D82FC92F20919202283010F0C4DF83
:101CB00020E0E22FF0E0EE0FFF1FEE57FD4FD08344
:101CC000C1832F5F20939202DF91CF910895CF932C
:101CD000DF93FB018FEF9FEF44305105B0F0D081CF
:101CE000C181AADFD093C404C3708091C5048C7FE6
:101CF000C82BC093C5046091C4047091C50484E0EE
:101D000090E00E94C83380E090E0DF91CF91089589
:101D1000AAE2B0E0EEE8FEE00C94343380EE91E00D
:101D2000FC0101962091F100208321E0883E92077A
:101D3000B9F78091E101893009F457C0C8F48230C5
:101D400009F4B2C0833009F482C0813081F18091FE
:101D5000E80083FFE6C08091E0019091E1019A30B4
:101D600008F0DFC0E92FF0E0EB51FC4C0C94083395
:101D70008A3009F489C08B3051F78091E0018132BB
:101D800031F78091E4019091E501892B01F7809171
:101D9000E800877F8093E8000ADC81E09091E2010F
:101DA000911101C080E08093100146DFD0CF809177
:101DB000E001813A61F68091E800877F8093E80036
:101DC0008091E4019091E501892B59F060E080E079
:101DD00090E070E093DB8091E8008B778093E800DF
:101DE000B6CF68E088EE91E0F4CF8091E0018132D7
:101DF00009F0ADCF8091E4019091E5018D7F892BB1
:101E000009F0A5CF8091E800877F8093E80080915A
:101E1000E80082FF17C09091F3008091F2000297D2
:101E200031F48091F100813011F0863021F48091FD
:101E3000F10080930F018091E8008B778093E80098
:101E4000B6DB85CF809151028111E1CF80CF8091A7
:101E5000E001813A09F07BCF8091E4019091E501A6
:101E6000892B09F074CF8091E800877F8093E80088
:101E70008091E80080FFFCCF809110018093F100F9
:101E80008091E8008E77DACF8091E001813209F00D
:101E90005ECF8091E800877F8093E80088DB8091A7
:101EA000E30180930E0153CF8091E001813A09F064
:101EB0004ECF8091E800877F8093E8008091E80012
:101EC00080FFFCCF80910E01D9CF803889F0823815
:101ED00041F58091E4018F70873018F58093E90017
:101EE0008091EB0085FB882780F91092E90006C0FD
:101EF00080912C02880F9091DD01892B9091E80050
:101F0000977F9093E8008093F1001092F100809108
:101F1000E8008E7723C0811116C08091E2018130E4
:101F200009F18091E80083FF0AC08091E800877F73
:101F30008093E8008091EB0080628093EB00AA968A
:101F4000E3E00C945033823061F78091E201811517
:101F500081F01092E9008091E800877F8093E8008B
:101F600026DBDFCF81E0933009F080E080932C0204
:101F7000F0CF8091E4018F702FEF280F263088F684
:101F80008093E9002091EB0020FFE3CF933031F400
:101F90008091EB0080628093EB00DBCF9091EB00AF
:101FA00090619093EB0021E030E0A90102C0440F62
:101FB000551F8A95E2F74093EA001092EA0080915B
:101FC000EB008860E8CF8111ACCF1091E2011F7760
:101FD0008091E3008078812B8093E3008091E8007A
:101FE000877F8093E800E3DA8091E80080FFFCCFF0
:101FF0008091E30080688093E30083E0111101C0C9
:1020000082E0809351028DCF8058823008F089CFD2
:102010008091E2019091E3018C3D53E0950791F5A9
:1020200083E08A838AE289834FB7F894DE011396AE
:1020300020E03EE051E2E32FF0E05093570084911E
:1020400020FF03C082958F703F5F8F708A30C0F091
:10205000895C90E08D939D932F5F243161F74FBF92
:102060008091E800877F8093E8006AE270E0CE010B
:10207000019644DA8091E8008B778093E80051CF95
:10208000805DE7CF292F33272330310509F44EC077
:1020900078F52130310509F488C08BE590E0EFE256
:1020A000F2E02230310509F03CCF2091E800277F93
:1020B0002093E8002091E6013091E7018217930711
:1020C00008F49C0140E02115310509F073C041116D
:1020D00071C08091E80082FDCDCF809151028115C1
:1020E00049F2853039F28091E80083FFF2CFC2CF08
:1020F0008091E4019091E5012132310509F446C057
:102100002232310509F00DCF8330910508F009CF57
:10211000FC01EE0FFF1FEF5DFE4F0190F081E02DFF
:10212000825E9E4FDC018C9190E010C09C013327B1
:10213000823021F12330310568F4232BB9F4E0EE2D
:10214000F2E0E4918E2F90E0E0EEF2E0009709F4E7
:10215000E8CEABCF2330310509F0E3CEECE9F2E075
:10216000E4918E2F90E0ECE9F2E0F0CFEEECF2E0BB
:10217000E4918E2F90E0EEECF2E0E8CFEAEBF2E0B3
:10218000E4918E2F90E0EAEBF2E0E0CF833091050E
:1021900008F0C7CEFC01EE0FFF1FE95DFE4F019076
:1021A000F081E02D89E090E080CF82E190E0EAE8E4
:1021B000F2E07BCF80915102811509F45BCF85302D
:1021C00009F458CF8091E80083FD54CF8091E80056
:1021D00082FD7FCF8091E80080FF75CF9091F30062
:1021E0008091F2002115310519F08830910550F0E9
:1021F00041E0089709F040E08091E8008E778093F5
:10220000E80061CF44914093F100319621503109AB
:102210000196E8CF803809F084CE8091E800877F6E
:102220008093E8008091DE018093F10070CE8111EF
:1022300078CE1091E201123008F073CE8091E80060
:10224000877F8093E8001093DE01B1D91115D9F092
:1022500084E08093510242E061EC81E025DA42E2C1
:1022600061EC84E021DA42E261EC82E01DDA42E2D4
:1022700060EC83E019DA80915102843051F482E0FD
:10228000809311014ECE8091E30087FDE1CF81E084
:10229000E0CF81E0F5CF80911301877F8093130118
:1022A00080911D03811103C082E00E94410580914D
:1022B000130184FF06C08F7E8093130182E00E9489
:1022C00033058091130185FF06C08F7D8093130134
:1022D00080E20E94330562CBCF92DF92FF920F9390
:1022E0001F93CF93DF93EC018B01F42E80911301A8
:1022F00082FF61C0C0902C04D0902D04CC16DD0666
:1023000019F0209709F057C0809113018B7F8093BB
:102310001301C1E081FD10C080912A0490912B042B
:102320009801281B390BC1E080910C0190910D019F
:102330002817390708F4C0E080911301C0FB81F928
:10234000809313016C2FC6010E94380880914004CD
:1023500081FF08C08091130180618093130182E0A6
:102360000E9439058091400485FF08C080911301C7
:1023700080628093130180E20E9439056C2FC601B0
:10238000F3DBF11431F08091B70485FF02C086FFC2
:1023900025C08091BA049091BB042FDA80912C045F
:1023A00090912D049C0130522115304308F4992757
:1023B0000DDC71DF0FC0CE01905281159043B0F457
:1023C000CE01992703DC80912C0490912D04C8172D
:1023D000D90779F310932B0400932A04DF91CF914E
:1023E0001F910F91FF90DF90CF900895CE01EACF1B
:1023F000CF93DF93EC014A855B856E857F850E94D4
:10240000CC088B810E9441058C810E943905C6DA77
:1024100086E0FE0111928A95E9F7DF91CF91089548
:10242000CF93DF93EC018D8181FD13C082608D839A
:10243000809143049B81892B809343048C810E946B
:102440003305ACDA488559856E857F85CE010E94BB
:10245000CC0810922704109226048D8180FD02C0C2
:10246000CE01C6DFDF91CF9108951F93CF93DF9305
:10247000182FA0919C03B0919D03109709F449C0B7
:1024800010929F0310929E03109222031092210338
:102490001696CD91DC911797CE019A9581159F41A3
:1024A00008F4D07ED1E0C11101C0D0E01996ED91C1
:1024B000FC911A97309731F01B966D917C9180E0DA
:1024C0000995D823D11539F08CEF8C0F813A28F576
:1024D0008C2F0E9464091115A9F0E0919C03F091E2
:1024E0009D03808584FD0EC080919B03811551F072
:1024F000808191819C01215031092F333E4710F496
:102500000E943C0A4BDA10929D0310929C03109299
:102510009B03DF91CF911F91089540DA8C2F32DB1E
:10252000DACF0F931F93CF93DF930CE914E0C1E848
:10253000D2E0CE010E949233F80161918F016817B9
:1025400019F0CE010E94AE332196C93AF2E0DF07BE
:1025500081F7DF91CF911F910F9108950F931F93F2
:10256000CF93DF930CE914E0C1E8D2E0CE010E94E2
:102570009233F80181938F012196C93AF2E0DF0787
:10258000A9F7CAE1D4E0FE0185919591009711F079
:10259000FC0109952C96F4E0C63EDF07A1F7DF9118
:1025A000CF911F910F910895ECE9F4E0128E138EF4
:1025B0008FEA90E09183808385E0848F28E833E17F
:1025C0003383228322E330E0378B268B28EC30E004
:1025D000318F208F158E35A324A3178E168E20E5FC
:1025E00030E031A320A382A317A216A29ADF24DB36
:1025F0001092C5041092C40480E084608093C504E6
:1026000060E074E084E090E00E94C833A7CF0F93AD
:102610001F93CF93DF93843030F5653020F54F3032
:1026200010F5C42FD0E0CC0FDD1F2EE1629FC00D4E
:10263000D11D112436E9839FC00DD11D1124CE0177
:1026400089960E949233082F10E0102F0027CE01A8
:102650008A960E9492339801282BC901DF91CF916D
:102660001F910F91089580E090E0F8CF462F672FDB
:102670002091540230915502232B81F4703F39F49C
:10268000403F61F480915202909153020895753059
:1026900028F44F3018F4843008F4B9CF80E090E08B
:1026A0000895A0E0B0E0E7E5F3E10C9430337C015D
:1026B00000913F0480913E04082BC3E0D0E010E07D
:1026C000C8010C2E02C0959587950A94E2F780FD0B
:1026D00009C02197A8F7D12C8D2DCDB7DEB7E7E043
:1026E0000C944C33DC2EB7018C2FC0DF0E944706C0
:1026F000019779F3F1CFCF93DF93D82FC92FD1DF93
:102700006D2F7C2FB3DF0E944706DF91CF91089594
:10271000FC018481811561F087819085009721F00B
:102720000E9447060C94D20380819181E4DFFACFA6
:1027300080E008951F93CF93DF93182FD92F611551
:1027400089F0411579F0ADDFC82F682F812F9D2FBB
:102750000E941404612F7D2F8C2F88DFDF91CF9191
:102760001F9108950E944A04C82FF4CFFC01462F00
:1027700087819085009721F4658180819181DACFEE
:102780000895382F292FCB01A32FB22F8738910519
:10279000A105B10520F487589C4F0C94923380E03A
:1027A000089585E290E00E949233893C89F486E2A4
:1027B00090E00E9492338E3359F487E290E00E94B9
:1027C000923391E08A3409F090E0892F8170089566
:1027D00080E0FCCFAAE0B0E0E0EFF3E10C942A3314
:1027E000C0904F02D090500281E090E09093500250
:1027F00080934F02812C912C10E0540100E019C00D
:1028000021E030E0123020F4F701859195919C0190
:10281000472D602F812F9BD8739422E0E20EF11C8C
:102820003FE07312EDCF0F5F8FE0A80EB11C0530B3
:1028300049F0C501880F991FFC01EC51FD4F7F0144
:10284000712CDECF1F5FFBE48F0E911C1430A9F6B4
:10285000ABDE1A8219821C821B821E821D821886A0
:102860001F8288EC90E09A87898709EA12E09E012E
:102870002F5F3F4F79014AE050E0B801C7010E9445
:10288000CC33065F1F4F093F32E01307A1F789E001
:10289000F70111928A95E9F78FEF9FEF9E838D8361
:1028A00087E08A874AE050E0B801C7010E94CC3334
:1028B000065F1F4F0934F3E01F07A1F786E0F70119
:1028C00011928A95E9F746E050E0B801C7010E94ED
:1028D000CC330A5F1F4F0937F3E01F07A1F7D092EF
:1028E0005002C0924F022A96EDE00C944633AAE0C3
:1028F000B0E0EDE7F4E10C942D3303E213E089EF4F
:10290000E82E82E0F82E97E0B92E28E1C22E22E0D0
:10291000D22EAA24A3944AE050E0B701CE0101963A
:102920000E948233F8013896DF018B2D1D928A9523
:10293000E9F789819A81D80111969C938E938F81B2
:1029400012968C9312978D8113968C93139788858A
:1029500014968C931497898515968C9315978B8173
:102960009C8117969C938E9316978A8587FD04C049
:102970001E96DC92CE921D9780FF02C0F801A086C1
:1029800081FF07C0D80118969C91189792601896FD
:102990009C9382FF04C0F80190859460908783FF28
:1029A00007C0D80118969C911897986018969C9328
:1029B00084FF04C0F80190859061908785FF07C06F
:1029C000D80118968C911897806218968C93BAE06B
:1029D000EB0EF11C015F1F4FE9E4EE16E3E0FE068B
:1029E00009F099CF2A96EAE00C944933A6E0B0E0CA
:1029F000ECEFF4E10C9430330DEB12E089E4E82EB7
:102A000083E0F82E98E0D92E46E050E0B701CE01E1
:102A100001960E948233F8018D2D11928A95E9F773
:102A2000B8016C5F7F4F89819A810E948307F8010A
:102A300091838083B8016B5F7F4F8B819C810E9463
:102A40008307F801938382838D8186838E818783B8
:102A5000F6E0EF0EF11C085F1F4F89E7E81683E0F0
:102A6000F80691F62696E7E00C944C33282FCB011C
:102A7000283070F44AE0249F90011124B901675571
:102A80007D4F4AE050E00E94823380E090E008955C
:102A90008FEF9FEF0895AAE0B0E0E1E5F5E10C9437
:102AA00035339C0197558115914068F4BE016F5FE5
:102AB0007F4F822FDBDF892B31F489859A852A9617
:102AC000E2E00C9451338091B4049091B504F7CFB7
:102AD000A0E0B0E0EEE6F5E10C943033162FD72FEE
:102AE000C42FD22E8115A9F0409337040E94930978
:102AF0009093DC018093DB01C77081E001C0880FF7
:102B0000CA95EAF70E94220DCDB7DEB7E7E00C9434
:102B10004C3390913704491336C0E090DB01F090BC
:102B2000DC010E9493099C012E193F097901812F34
:102B30009D2FB1DFE816F90630F5D0E2DD0DCD1599
:102B4000A1F0C77011E0812F01C0880FCA95EAF784
:102B50000E94300DD83048F48D2D877001C0110FC0
:102B60008A95EAF7812F0E94220D802F5AD8D830FB
:102B700058F62D2D277081E001C0880F2A95EAF7BD
:102B80000E94300DC1CFC77081E001C0880FCA9587
:102B9000EAF7F6CF9C01CB01BA01F9013296E49134
:102BA0004E2F50E06E17710548F0F901349665918B
:102BB00075910E94723380E090E008958FEF9FEF4F
:102BC0000895A4E0B0E0E7EEF5E10C9432338B0118
:102BD000FC013396F49019821A821B821C82452BC9
:102BE00031F48FEF9FEF2496E5E00C944E3344E0F0
:102BF00050E0BE016F5F7F4FCDDF019691F381E022
:102C000090E00F2C02C0880F991F0A94E2F7092E5A
:102C1000000CAA0BBB0B49815A816B817C818423F8
:102C20009523A623B72321E0892B8A2B8B2B09F42C
:102C300020E0F801208380E090E0D5CF9C01CA011C
:102C4000F9013296E4914E2F50E08E17910550F025
:102C5000F9013496859195910E94723362DC80E08F
:102C600090E008958FEF9FEF0895A4E0B0E0EBE3CC
:102C7000F6E10C942E337C016B01CA01F701339607
:102C8000B49019821A821B821C82892B31F48FEF37
:102C90009FEF2496E9E00C944A3344E050E0BE01F3
:102CA0006F5F7F4FC70176DF019689F381E090E087
:102CB0000B2C02C0880F991F0A94E2F7809590951B
:102CC000092E000CAA0BBB0B49815A816B817C81B8
:102CD00084239523A623B723F6012081022F0170B8
:102CE00010E00B2C02C0000F111F0A94E2F7012E16
:102CF000000C220B330B802B912BA22BB32B89833F
:102D00009A83AB83BC8344E050E0BE016F5F7F4F8A
:102D1000C70194DFBECFAAE0B0E0E1E9F6E10C9490
:102D20002933FE0131968AE0DF011D928A95E9F789
:102D30009DE2A92E91E0B92E8F013F01EE24E3948C
:102D4000F12C31E4C32E31E0D32EF50181915F01E6
:102D50008F3F09F444C0F894E82FE295EF70F0E05B
:102D600021A18F70A70102C0440F551F8A95E2F779
:102D7000CA01922F982B91A392A18095892382A3B7
:102D8000789400C0E2E3F1E021E030E0812C912C66
:102D900041914F3F79F0A42FA295AF70A05EB0E0B3
:102DA0008C9190E04F7002C0959587954A95E2F717
:102DB00080FF3BC080E090E0882A992A220F331FD1
:102DC000CE16DF0629F7F50182918F3F11F00E94A0
:102DD000450750EA5A95F1F7D8018D929C920E5F03
:102DE0001F4FB2E3AB16B1E0BB0609F0AECF4AE02D
:102DF00050E0B30181E292E00E946533892BB9F083
:102E00008AE0F301A1E2B2E001900D928A95E1F728
:102E100081E08093DA010E9493099093D901809315
:102E2000D8012A96EEE00C944533C901C5CF8091B4
:102E3000DA018115B1F30091D8011091D9010E94F6
:102E40009309801B910B059760F34AE050E061E223
:102E500072E085E492E00E946533892B49F08AE0B4
:102E6000E1E2F2E0A5E4B2E001900D928A95E1F78B
:102E70001092DA01D6CFA0E1B0E0E1E4F7E10C94E2
:102E80002733FE01319680E1DF011D928A95E9F733
:102E900009E010E099E7A92E93E0B92E27E8422E29
:102EA000512C612C712C4F0173016201B1E14B1661
:102EB0005104610471041CF080E1C82ED12CA601DC
:102EC000B501C4010E949F33AC0CBD1C0D2C000C3D
:102ED000EE08FF084C185D086E087F08015010408E
:102EE00019F76096E0E10C9443336FEF85E290E0D0
:102EF0000E94AE336FEF86E290E00E94AE336FEF38
:102F000087E290E00E94AE3360E088E290E00E94A9
:102F1000AE3360DCB0DF69EC85E290E00E94AE3356
:102F20006EE386E290E00E94AE336AE487E290E0CE
:102F30000C94AE33A0E0B0E0E0EAF7E10C942E335D
:102F4000EC0188818115F1F0813009F042C089815E
:102F5000813029F48A8123960E94110EF2CF8230AB
:102F600029F48A8123960E94430DEBCF833029F404
:102F70008A8123960E94C20DE4CF843041F02296CC
:102F80008111DFCFCDB7DEB7E9E00C944A338A81F7
:102F9000239620E030E09AE0682F6053770BAB0176
:102FA0006A30710560F02115310551F3EFE9FFE05A
:102FB0003197F1F700C0000021503109F4CF929F02
:102FC000B001939F700D11249A01260F371F89912C
:102FD000E3CFE82FF0E0E155FE4FB490282F26957F
:102FE0002695269530E0F901E156FE4FE490877072
:102FF000F12C082E02C0F594E7940A94E2F7E0FA67
:10300000EE24FF24E0F8F901E157FE4FC490D12CE3
:10301000082E02C0D594C7940A94E2F7C0FACC24D3
:10302000DD24C0F8F901E158FE4F049110E002C020
:10303000159507958A95E2F701701127E114F104BF
:1030400019F081EE0E94430DC114D10419F086EEEF
:103050000E94430D60E070E08B2D0E94FB0DC114B7
:10306000D10419F086EE0E94C20DE114F10419F0AA
:1030700081EE0E94C20D0115110519F08CE20E942B
:10308000110E21965ECFAEE0B0E0E9E4F8E10C94D9
:1030900025337C01DC0114968C91811509F4BCC1A7
:1030A00060E0C70163DB9C01F7018681803170F429
:1030B00040914A0490914904491333C09091980477
:1030C000911521F090919904903158F1D7011596FE
:1030D0009C91911110C02115B0E53B0708F084C008
:1030E0002115E0E23E0708F094C0283E310590F437
:1030F000203E3105B0F43093B2022093B102D701E3
:1031000012968D919C91909348048093470410925D
:10311000140107C0C9019A9581159F4160F72111DB
:10312000EACF61E0C70122DB8C01F70185818115BF
:1031300021F180912604909127040097F1F008175F
:103140001907D9F0FC01FF27887F9927892B09F0FF
:1031500062C084E0EE0FFF1F8A95E1F7EA55FC4F4D
:1031600085818460858311830083CF0159D91092B2
:10317000430461E0C701FADA8C01809112038111E6
:1031800051C0D70115968C91811509F4FBC001152A
:10319000B0E51B0708F0E1C00115E0E21E0708F0EA
:1031A0003FC10115F7E01F07E9F1C0F5C801805ED6
:1031B00091090897B8F1309140048091430420911F
:1031C0003C0499E0F701AEEFB2E001900D929A95C0
:1031D000E1F7109306030093050310920803832B75
:1031E000822B8093FD021EC0203E42E5340760F42E
:1031F000203852E5350708F094CFC9018052924536
:10320000809708F078CF8DCFC90187579C470297E8
:10321000F8CF8031F6CFE0E0F0E0A2CF01153FE03B
:10322000130749F6F70185818111F7C1011527E5DB
:10323000120708F401C3011538E5130710F00C94C8
:103240005F24680147E5D41A63E173E08C2D0EDC3E
:10325000892B31F5C601F4E0880F991FFA95E1F743
:10326000FC01EA55FC4F2281213009F0B5C22091C2
:10327000130330911403232B99F0209115033091FF
:103280001603232B69F02091170330911803409106
:10329000190350911A03242B352B232B09F4A6C2B2
:1032A00080911D03811509F441C3C0904004D09062
:1032B0003C040E94930988579C4E90931F0380936F
:1032C0001E03D70115968C91811509F42FC38D2DFE
:1032D0008C298D79811153C30115B0E51B0708F0C6
:1032E00001C30115E0E41E0708F050C3063E1105B6
:1032F00009F41CC3C80190528115904208F007C31D
:10330000D70116968C91803108F433C36801DD240F
:103310008091130180FF46C38DEF0E944105BDE2FD
:10332000CB16D104A1F008F050C3F8E2CF16D104B7
:1033300008F03AC32EE1C216D10408F039C334E0D4
:10334000C31AD1084AE1C416D10408F018C3809109
:1033500043048260809343042BC3003E42E514077C
:1033600050F4003652E5150708F05CCFC8019255BD
:10337000803491051FCF980127573C4725303105F0
:1033800008F019CF0937BCE71B0709F04EC02091A0
:10339000050330910603232B79F18115A1F081E01B
:1033A0000E94A6088091FD020E94270D89E0EEEFA1
:1033B000F2E0A4EBB2E001900D928A95E1F78091E2
:1033C00008038093B30286E0F701A4EBB2E001901A
:1033D0000D928A95E1F78091B3028093120384EBFA
:1033E00092E051DE10921203F7018581811104C031
:1033F0008091FD020E94350D8091440487708115F3
:1034000059F0F7018581811539F08091C50482FF5B
:1034100003C082E00E9418052E96E2E10C9441332D
:10342000D70116968C918031C5CE0A37FCE71F076D
:1034300009F0F8CE811509F4C5C0A0900503B0903D
:1034400006032091FD022F832983BE016F5F7F4F0A
:10345000C5010E9483072C0139813D87BDEBCB2E2E
:10346000B2E0DB2E01E010E022242A94D601179668
:103470003C90179733FE53C06D907C901197129635
:103480008D909C90139746145704B9F41496BC91F0
:10349000BB87232DF60146816B2F8D850E949D07EA
:1034A000811559F08B850E94BC03281634F4D6018F
:1034B00015969C918401192B282E48145904C9F49F
:1034C00031FE17C0F601F581FB87232DD601169634
:1034D0004C916F2F8D850E949D07811551F08B8532
:1034E0000E94BC0328162CF4F60194818301192B49
:1034F000282E30FE14C0FFEF2F1211C0013011052D
:1035000071F4232DD60116964C9160E08D850E94B2
:103510009D07811521F0F60185818401182BF8E0C3
:10352000CF0ED11C2DEF32E02C153D0509F09ECFBA
:1035300001301105E1F58F8182958F703F81832BDA
:103540008F7011E0303108F410E01295107F182BC5
:10355000A11440E2B40620F5A11451E0B50608F02C
:1035600055C00A2D812F8D704A2D811509F451C047
:103570006AE085E996E00E94B708282F30E021151F
:10358000310551F4402F66E187E796E00E94B708C5
:10359000282F30E0811549F0F901F12B8F0107C088
:1035A000C50190528115904390F100E010E087E052
:1035B000E9E0F3E0DF011D928A95E9F7109311032A
:1035C000009310038091100390911103892B09F44B
:1035D00013CFF7018581811539F08FEF0E94A6087E
:1035E000809108038093070386E0F701A9E0B3E028
:1035F00001900D928A95E1F7809107038093120361
:1036000089E093E040DD10921203F6CE1B29BB2423
:10361000A8CF68E08DE896E0AECFC8019757803814
:10362000910508F0EEC0003108F0E6CE66E870E0E3
:1036300080E090E0A6D88111DFCE812C912C54013E
:10364000011143C004E0AE014F5F5F4F6A01D60134
:10365000E02F1D92EA95E9F724013501FFEF4F1A9B
:103660005F0A6F0A7F0AC501B4018BD8898381156F
:1036700009F4C2CE813009F0ACC0A50194012E5FDF
:103680003F4F4F4F5F4F2F83388749875A87C3017A
:10369000B20177D8182F8A83811509F4ADCE8FEF48
:1036A000810F833050F56F81788589859A8569D837
:1036B0008B83811511F0C6013DDC2401350133E017
:1036C000430E511C611C711C46C0F7E88F16910413
:1036D000A104B10409F490CEC501B40152D82FEF72
:1036E000821A920AA20AB20A8111EFCF0150A8CF22
:1036F0004F80588469847A842EC08BEF810F833089
:1037000098F52401350143E0440E511C611C711CE5
:103710006F81788589859A8534D88B838115D9F016
:10372000C301B2012ED88C83811571F08B819C81ED
:1037300081305FEF950710F0982F8827163071F0D1
:10374000173079F00E94012A2401350154E0450E1A
:10375000511C611C711C5301420179CF0E94BF2989
:10376000F3CF0E94E029F0CF143009F0C1CF6F8170
:10377000788589859A8505D8182F2401350184E03C
:10378000480E511C611C711CC501B4016D5F7F4F57
:103790008F4F9F4F0E94C113111509F42DCE811533
:1037A00009F42ACE8150990B4FEF489F9001499F11
:1037B000300D1124A12FA150BB0B2A0F3B1F21500C
:1037C000310948F2EFE9FFE03197F1F700C000005E
:1037D000F6CFC601AFDBBFCF223009F061CD20911B
:1037E000170330911803232B09F45ACDFC01E5553A
:1037F000FC4F20812E7F20838A559C4F0E941012FF
:103800004FCD03375CE71507B9F480911D0381158F
:1038100019F00E943A0DF0CD109240040E94490523
:103820000E94930988579C4E90931F0380931E0318
:1038300081E080931D03E0CD023A82E51807C1F1D3
:1038400058F4C80190528115904220F1013E1105B3
:1038500079F1053E110503C0023BB2E51B0709F0F3
:103860001FCD25EE30E02770332781E090E001C0C6
:10387000880F2A95EAF72091200330911D03311516
:10388000F9F0D70115963C913115A9F0282B20931A
:103890002003B2CDF7018681803108F001CD812F60
:1038A00099278F7199278230910511F04297D7CFD0
:1038B00021EE30E0D8CF80958223809320039CCDE9
:1038C000322F3823311509F4EBCC982F90959223A1
:1038D000909320030E943905F7018581811509F431
:1038E0008BCDDECC003EB2E51B07C0F4003CE2E528
:1038F0001E07E0F4003AF2E51F0758F4003622E50F
:103900001207A0F4C80192558034910578F068013F
:10391000FFCC043B32E5130749F0F9CF09374CE7F8
:10392000140718F507375CE7150788F3D7011596D4
:103930003C90311409F456C00E35BCE71B0709F45E
:103940004DC00F35ECE71E0751F00D35FCE71F07A2
:1039500009F048C080911201811509F43FC010920E
:10396000120180E00E94351247CD0B378CE7180713
:10397000D3CF812F8F718431C9F2863171F00E94CB
:103980003A0D809120030E943305D0CFD7011696BF
:103990008C91803108F0BACCC9CF76EEC72E72E197
:1039A000D72EB6CC8FEFB9CC5AE2C516D10439F771
:1039B00080912003811531F08091430492E08927A2
:1039C000809343040E94CE0CB1CF8CE4C816D1047E
:1039D00079F39DE2C91692E0D906E9CF81E08093A0
:1039E00012010ACD80911201811149C0C801975579
:1039F0008115914008F0DFC05801F8EFAF22BB24D9
:103A0000A114B10409F0F8CCF801FF2754E0EE0F3F
:103A1000FF1F5A95E1F79F012A553C4F6901D701D5
:103A200015968C91E555FC4F908180FB90F9908321
:103A3000811509F412C20E9493099093290480937E
:103A40002804F60182818F5F8283809143049091E4
:103A50004004892B838380913C0484834681578171
:103A600066857785C6010E94CC08D60115968C9193
:103A700081FF5801B0922704A09226049CC038010F
:103A800030EE631A710850903D0480914004582A2A
:103A900080913C04582A48E06416710408F05EC026
:103AA00098012770332781E090E001C0880F2A95A4
:103AB000EAF7311409F44FC0582AD7018D919C912F
:103AC0000E944A0421E030E0F90102C0EE0FFF1F1E
:103AD0008A95E2F7FC87EB8720919C0330919D0348
:103AE00038872F834091A4035091A5035E874D87AB
:103AF00063E2C62E63E0D62EA12CB12C511005C076
:103B0000D60112968C9181111BC0F601838190E041
:103B10002B853C8582239323892B91F08085982FD8
:103B20009770911101C087E038E06316710408F0C6
:103B3000BFC0311409F4B8C0869581708111BDC031
:103B40009FEFA91AB90AAFE0CA0ED11CB8E0AB16B4
:103B5000B104A1F61CC080955822AFCF311091C09E
:103B60008091A4039091A5030817190781F410927E
:103B7000A5031092A4031092A0031092A103109227
:103B8000A2031092A30310929F0310929E038091B0
:103B90009C0390919D03009709F428CFE8E06E16EE
:103BA000710408F044C1652D0E945E08811103C0B4
:103BB00081E00E9435128091B70480FFBEC10E944F
:103BC00093095C01F7018581811509F4C8C18091D1
:103BD000130182FF06C040E0B50180E090E00E9442
:103BE0006C110431FCE71F0709F4B5C105312CE75E
:103BF000120709F44FC103313CE7130709F490C1E0
:103C0000C80190528115904308F04EC110922D04C6
:103C100010922C04F701958191111092370406310E
:103C2000FCE71F0709F06EC2809140043091B60492
:103C300030FF04C0282F2474211158C2282F2A7A5B
:103C400031FF04C0482F4171411120E032FF04C010
:103C5000482F4878411120E033FF03C08272811160
:103C600020E0911509F444C281E0211101C080E0F7
:103C70008093380485E3211101C089E20E94300954
:103C8000C7C01093A5030093A4030E94300A609359
:103C9000A0037093A1038093A2039093A3031092B7
:103CA0009F0310929E0309CF82FB882780F946CF9D
:103CB000311409F445CF80FF43CFD6018D909C90FD
:103CC0000815190519F4311409F43ACFEF81F88574
:103CD000EC15FD0509F434CFD6011D96ED91FC914C
:103CE000309721F08081811509F42ACF652DC60116
:103CF0000E945E08811509F423CF81E0081519059B
:103D000009F080E0482E43208114910441F04110D5
:103D100006C0ED85FE858E169F0609F011CF80E066
:103D20000E943512D0929D03C0929C0381E0809343
:103D30009B038FE08A9DF0018B9DF00D1124ED5DBA
:103D4000FC4F85818093220341100EC081149104A1
:103D500059F0808191819C0124503109213A31052B
:103D600008F049C00E9464098FE08A9DF0018B9D94
:103D7000F00D1124ED5DFC4FC680D780C6019A95E9
:103D800081159F4110F420EED22299249394C6010C
:103D900001978F339E4708F0912C8FE08A9DD001C8
:103DA0008B9DB00D1124AD5DBC4F1996ED91FC912A
:103DB0001A97309731F01B966D917C9181E00995AF
:103DC00098229114A9F08FE08A9DF0018B9DF00D4F
:103DD0001124ED5DFC4F868197810E9489038093B9
:103DE0002103C60148E06416710440F40E943C0AB5
:103DF0000E94CE0C0AC00E94C20DB6CF0497813A31
:103E0000910548F48C2D0E943009411409F4EECD3F
:103E10000E94CE0CF1CA0E94CE0C8FE39CE9019760
:103E2000F1F700C000008C2D0E94430DEECFDC01A5
:103E30002D913C910217130741F4311009C01092E3
:103E40009B0380E00E943512D1CD311409F4CECD10
:103E5000FC01808585FDCACDF4CFF90144855585E7
:103E600066857785C9010E94CC08D60115968C918C
:103E700081FFA1CEC6010E94F81180912604909185
:103E800027040817190709F096CE109227041092FC
:103E9000260491CE90911301892F8E7F90FF81602F
:103EA000809313010E944B118091130180FF45C044
:103EB0000832110508F069C00E31110508F076C00E
:103EC000C80104974A9788F58091B70484FD2DC0F6
:103ED000D70115968C91811509F4D6C080913C04C8
:103EE00090914004892B8D7F811509F464C0109254
:103EF0002D0410922C048091B70481FD5CC060E019
:103F0000C8010E94380860E0C8010E94B40D809189
:103F10003C048D7F0E941D0A82E00E9418056CCA35
:103F200080911301816080931301F70185818115D0
:103F300021F010922D0410922C04D70115968C912B
:103F4000F801E851FC47E730F10508F063CEE15194
:103F5000FC4C0C940833809113018E7FA1CF80918B
:103F600013018F7E013E110531F0053E110531F43C
:103F7000809113018F7D8093130196CFC8019052D9
:103F80008115904308F090CF45CE0933110558F4C0
:103F90000D32110518F40B32110539F68091B70472
:103FA00082FDC3CF95CF04361105F7CF8091B704BA
:103FB00083FDBBCF8DCF89E0F701AEE2B4E0019085
:103FC0000D928A95E1F7109231041092300480919D
:103FD0002C0490912D0408171907C9F52091B704F6
:103FE00025FF35C03091130131FF02C026FF2FC0DD
:103FF00020912A0430912B046501C21AD30A0E9431
:104000004B15C816D90618F58091400481FF08C0E9
:104010008091130180618093130182E00E94390531
:104020008091400485FF08C08091130180628093D5
:10403000130180E20E943905609113016695617059
:1040400080912C0490912D040E94B40DD5C98091CB
:104050003C04D0904004D82AD1FADD24D0F88D7FDA
:104060000E941D0A10932D0400932C04B0922B047F
:10407000A0922A04DD0C6894D2F890911301997FE4
:10408000D92AD092130148CF40E0B501C8010E945F
:104090006C11B2C906E221EE41EE6AE17CE70E94B2
:1040A0006815AAC907E225EE45EE6BE17CE7F7CF7C
:1040B00006E221EE40EE68E17CE7F1CF07E225EE73
:1040C00044EE69E17CE7EBCF06E221EE42EE6CE1E3
:1040D0007CE7E5CF07E225EE46EE6DE17CE7DFCF3A
:1040E00008E221E045EE6EE17CE7D9CF20E0A8CDE3
:1040F00080913804811521F085E30E94640988CEFF
:1041000089E2FBCF07372CE71207F9F008373CE7C5
:10411000130731F19801205E32452032310528F530
:10412000911123C00F7181E090E0AC0102C0440FF7
:10413000551F0A95E2F78A01642F83E090E00E9400
:10414000AE33802F0E94F60357C981E0911551F0DC
:104150000E94FC0343E062E081E00E947E044CC9BF
:1041600082E0F4CF0E940604F5CF4091390480919B
:104170003F04282F30E02095309570E0242337232A
:10418000232B19F04823409339040B375CE71507BC
:1041900041F4911509F430C90E94BF030E947F08C1
:1041A0002BC9003482E5180708F056C00032A2E59A
:1041B0001A0708F058C00115B0E51B0758F501159E
:1041C000E0E41E0708F065C0911509F47BC00A35CC
:1041D000BCE71B0709F4FBC008F0DFC00130FCE7B7
:1041E0001F0709F4F2C003302CE7120709F4E7C0F7
:1041F00001153CE7130709F065C00E941C0E8FEF04
:1042000094E3ACE081509040A040E1F700C0000092
:104210000E940B0C9801305521153240A8F69801E8
:1042200045E0369527954A95E1F7822F8F702091CA
:10423000390430E041E050E0082E02C0440F551F21
:104240000A94E2F724233523232B09F4BDCF9111DF
:10425000A5CF10924004DCCD9801205C324520327D
:10426000310508F0B1CF802F8F712091390430E0F3
:1042700041E050E0082E02C0440F551F0A94E2F7B7
:1042800024233523232B09F49FCF911509F4B4C8B7
:1042900085CFD70116968C91803108F095CF91117A
:1042A00011C0212F2F7081E090E002C0880F991F6C
:1042B0002A95E2F72091390430E082239323892B59
:1042C00009F09AC8D70117968D919C91009709F42F
:1042D00082C00E944706082FD92E86E0F701DE0132
:1042E000119601900D928A95E1F7D7011596BC9031
:1042F00015971696CC90C2949FE0C92280914404F1
:104300008770811501F19B2CB114F1F08D2D807F08
:10431000803461F080E2800F8830A8F08D2D807E9F
:10432000803221F4023078F0C11469F08091C50424
:1043300082FF09C082E00E941805809144048770C2
:10434000992493948111912CAD2CA2948FE0A822F2
:10435000B8E0AB1609F481C1E9E0AE1608F08BC0F5
:10436000F4E0AF1608F04FC01D2D1F7022E0A2161A
:1043700008F494C08D2D807F803211F01295107F4B
:10438000011509F4BFC0013009F429C1B11409F4C1
:1043900035C1C11409F4D0C095C00B354CE71407E2
:1043A000C1F08091C504002482FF0394802D0C3558
:1043B0005CE7150709F086CF0E94910C83CF6FEF61
:1043C0007FEF80E090E00E94C8330E943A0E81E0C7
:1043D000F3CF80E0F1CFF7018581C080D1808115D6
:1043E00069F0C6010E945113182F682FC6010E9460
:1043F0001404B601812F0E9436136BCFC6010E94B0
:104400004A04182FF6CF34E0A31609F409C1AA2DE7
:10441000A850BB0B149718F40E94D108912C802F40
:104420009D2D0E94D203811541F0B11409F41CC2E4
:10443000C11409F410C21092C8049114B1F0809113
:10444000440480FD12C0D70115961C92869586956E
:1044500086950E94FC03C7010E9443188091440482
:104460008695869586950E94060460E0C7010E94A5
:10447000B6130C940C1A49E0A41609F45DC186E049
:104480008A0D8F70823018F6023F09F065C18D2DBC
:104490008F71B1105EC10E94FC03B9CF50E1D516F7
:1044A00010F01295107FB114B9F0111559F080E297
:1044B000800F883010F0011109C0812F0E94330550
:1044C0000E94CE0C802F0E94430DA1CF8091430407
:1044D000812B80934304F4CF802F0E94C20D1115CD
:1044E00009F495CF80E2800F883010F0011104C0EC
:1044F000812F0E94390503C0812F0E9441050E942F
:10450000CE0C85CF8091C50482FD12C0B11449F054
:10451000111529F0812F0E9433050E94CE0C80E0F6
:10452000D2CF80E00E94C20D111509F470CFE0CF08
:10453000B11491F1C11004C0812F0E94220D67CFE8
:10454000B1E0CB1211C080903C04812F8821181754
:1045500009F45DCF0E94930990933B0480933A0441
:10456000812A80923C0453CF8091B804823008F4B1
:104570004ECFC8124CCF812F0E94220D812F0E9456
:10458000080A80913D04912F9823191709F43FCF11
:10459000812B80933D043BCFC11012C0812F0E941C
:1045A000300D812F0E94080A80913D04912F98239D
:1045B000911509F42CCF1095182310933D0427CFA3
:1045C0008091B804823008F422CFE1E0CE121FCFF0
:1045D000809140048123811509F419CFDFCF8091A8
:1045E000BE04B11421F08C1508F411CFA5CFC81664
:1045F00008F00DCF812F0E94300D09CFC114D1F3E7
:104600008091BC049091BD04093321F08091BA04DB
:104610009091BB040E94FD0B802F0E94C20DF7CE2B
:104620008D2D869586958370811569F0813009F00E
:10463000EECE802F9D2D9370B11002C080E090E0EF
:104640000E940809E4CE802F9D2D9370B11002C006
:1046500080E090E00E94E008DACE8D2D8370811119
:1046600033C0B110D4CE402F429546954770440FC9
:10467000440F802F8F70042E01C0880F0A94EAF730
:10468000202F207104FF07C02FE030E001C0220F6F
:104690004A95EAF720953D2D3695369533703230A0
:1046A00071F0333051F040913E04313029F0822BCB
:1046B00084230E94F603ABCE842B822BFACF822B6D
:1046C00090913E048927F5CFB11459F1D0FE9FCEC9
:1046D000402F429546954770440F440F802F8F70AE
:1046E000042E01C0880F0A94EAF7202F207104FFDE
:1046F00007C02FE030E001C0220F4A95EAF720956D
:104700003D2D369536953370323089F0333069F06F
:1047100040913F04313041F0822B84230E94F90301
:1047200076CE8230A8F673CE842B822BF7CF822BE5
:1047300090913F048927F2CF1D2D1F70B11429F0ED
:10474000812F0E94FC03802FF8CE802F0E94300D15
:10475000812F0E9406045BCE60F4003FB9F0013F58
:1047600081F0B11409F472C0C110ACCE8D2D8F71DF
:1047700092CE033FF9F0043FA1F78091C50482FD7A
:1047800025C08D2D8F71B11421F385CE8091BE048B
:10479000B11461F0C81608F03ACE2D2D2F7181E0CA
:1047A00090E001C0880F2A95EAF7C2CF8C1508F473
:1047B0002ECEF3CF80E0B11409F4B0CF81E09D2D6F
:1047C0009F7101C0880F9A95EAF7A8CF8091B8042D
:1047D000823048F1B114C9F090914404977094303C
:1047E00059F41092440410924604109245048D2D01
:1047F0008F710E94060410CE63E0C81608F00CCE3C
:104800008D2D8F710E94F40907CEC81640F01092CA
:104810004404109246041092450464E0F1CF81E014
:104820000E941805F9CDB11431F063E08D2D8F7120
:104830000E94F409ECCD81E00E941805F2E0CF1649
:1048400008F4E5CD82E00E941805E1CDC110D8CE74
:104850008D2D8F717ECF8091420480934104809191
:10486000400480934204E9CD40E060E089819A8170
:104870000E949A139C0110914004C11429F01092D7
:10488000C80410934204D9CD8091C6049091C70406
:1048900028173907B1F78091B90482FFF0CF8091D2
:1048A000C804811561F3809141040E94220D802F7C
:1048B0000E94110E809141040E94300DE0CF033719
:1048C000BCE71B070CC8A0E0B0E0E9E6F4E20C94FA
:1048D000303380919904803108F049C08091980468
:1048E000811509F444C0C0914A0489E0D82E809112
:1048F00049048C17E1F1EC2EF12CDC9EE00111242F
:10490000FE01E55BFB4F84818115B1F191818091BE
:104910009404981331C090818091930498132CC013
:104920008581811129C00281138180919504909124
:104930009604081B190B60E083E994E00E94B6130B
:104940000E944B1508171907B8F4809199048F70CD
:10495000806180939904CF5ADB4F88818F7080618A
:10496000888383E994E00E9443180E940E05CDB726
:10497000DEB7E7E00C944C33E7012196C770B7CF60
:10498000CF92DF92FF920F931F93CF93DF93182F55
:10499000092F89E0F82EC0914A0480914904C81774
:1049A00099F1FC9EE0011124CE01855B9B4F6C01C7
:1049B000FC018581811589F0C6010E94881381154B
:1049C00061F0FE01EF5AFB4F20812F7020612083A0
:1049D000F601808191810E944F0EC6010E9443180A
:1049E00020914A0430E02F5F3F4F277033272093F8
:1049F0004A04C55BDB4F89818013CDCF8881811349
:104A0000CACF8D81811539F2DF91CF911F910F911E
:104A1000FF90DF90CF900895EF92FF921F93CF9376
:104A2000DF93EC0120911401211541F010E0812F5A
:104A3000DF91CF911F91FF90EF900895EA80FB8066
:104A4000E61AF70A24EFE21621E0F20678F760E0B2
:104A5000CE010E94B6139C0130522115304330F72D
:104A60000E94D904811511F38091B1029091B20294
:104A70000E94D904182F8115C9F28091C204909127
:104A8000C304853F21E0920710F084EF91E0E8161F
:104A9000F90660F68E818F7080618E83888199819E
:104AA0000E944F0E0E949D04CE010E944318BFCF6A
:104AB000AFE0B0E0EEE5F5E20C9426338C0186E041
:104AC000F801DE011A9601900D928A95E1F7D8015E
:104AD0004C9011963C9011971296ED90FC90139784
:104AE00014965C90149715966C9061100CC05091C0
:104AF0009202252F30E0E0E08E2F0E2E000C990B55
:104B0000821793073CF153E9A52E54E0B52E80910E
:104B10009704811151C05114D1F0611409F419C3E3
:104B2000C8010E948813811509F413C360914704DA
:104B300070914804C80170DF811109C089E0F80153
:104B4000A3E9B4E001900D928A95E1F7BCDEFF2461
:104B5000F3948CC0880F991F8E579D4FDC011196DE
:104B60004C911197431103C08C91481611F0EF5FDF
:104B7000C3CFEF3F41F2D80116968C9116978F70F4
:104B8000806116968C93E517A0F4AFEFA50FA09364
:104B90009202EA1770F4F0E0EE0FFF1FEE57FD4FA0
:104BA000B0E0AA0FBB1FAE57BD4F8D919C91918372
:104BB00080830E949D04A7CF60E083E994E00E9477
:104BC000B6136C01709098048091950490919604AE
:104BD0004701881A990A60E083E994E0711409F4A6
:104BE0005CC20E94B6130E944B158816990608F005
:104BF0000FC2511409F4ABCF80919404F801918154
:104C0000B0909904F0E1BF1608F0C8C1981350C0E5
:104C100090919304D8018C9198134AC0611048C0B8
:104C20008B2D8F7080618093990483E994E00E94BA
:104C3000431880919904F8018683F0909504E090E0
:104C4000960449E0D42E00914A0480914904081743
:104C500051F0D09E80011124055B1B4FD8011596A1
:104C60008C91811108C00E940E05F12C8F2D2F967A
:104C7000E1E10C944233F801B280C380C8010E9484
:104C8000881381110EC0C8010E94431880914A0404
:104C900090E001968770992780934A04FB2CEC2CB6
:104CA000D2CF6F2D7E2DC801B7DE8111EFCFDBCFC4
:104CB000F0E2DF1AC11420E3D20608F084C06110CC
:104CC00005C140E0632D842D0E94DE0B81114FC091
:104CD00040E0632D842D0E94DE0BF82E811509F42F
:104CE00029C18091B90480FFC0CF83E994E00E947C
:104CF000431860E083E994E00E94B6138C01F090C1
:104D00004A047F2C98E0E92E23E9822E24E0922E9B
:104D100039E0432E809149047816A1F0A72CB12CDC
:104D2000479CC0011124FC01E55BFB4F6F0160E073
:104D3000CF010E94B613582E692ED60115968C917C
:104D4000811197C0B8E0EB1618F419E0EF10ACC071
:104D50008A859B8515DE0E949D040E940E0589E0D0
:104D6000E3E9F4E0DF011D928A95E9F77ECF60E088
:104D7000C8010E94B6138091B90483FFA9CFB8017E
:104D800083E994E00E94AA048111A2CF8091990442
:104D90008F70806180939904809193049091940422
:104DA0000E944F0E83E994E00E944318E3E9F4E087
:104DB00089E0DF011D928A95E9F78A859B85E0DD10
:104DC0000E949D0450CF611409F482CF8091990410
:104DD0008160809399048091B90481FF46CF83E973
:104DE00094E00E94431800914A04809149040817F6
:104DF00009F4CCC0E02EF12CB9E00B9FC0011124C6
:104E0000FC01E55BFB4F6F01CF010E948813811508
:104E100009F4BCC089E0F601A3E9B4E001900D9269
:104E20008A95E1F7C701019687709927082F80932B
:104E30004A040E940E0589E0F82E809149048017EB
:104E400009F411CFF09E80011124055B1B4FC801AE
:104E50000E948813811107CFC8010E9443188091D6
:104E60004A0490E0019687709927082F80934A049E
:104E7000E4CF10520115E0E31E0708F063CF8091E4
:104E8000B90483FD0AC0E72CC5010196F82FF7701D
:104E90007F2E052D162D46013DCFB601C4010E947F
:104EA000AA04811589F3EFCF1F9DC0011124855BF2
:104EB0009B4F0E94431820914A0430E02F5F3F4FE0
:104EC00027703327F22E20934A0440CF8091990413
:104ED00081608093990460E0C8010E94B6138091BC
:104EE000B90483FF78CFB80183E994E00E94AA0453
:104EF000811171CFF0909904E894F0F8F092990440
:104F0000C8010E9488138111B0CE8F2D8F708061EF
:104F10008093990480919304909194040E944F0E81
:104F20000E949D0483E994E00E944318E3E9F4E0C1
:104F300089E018CF8A859B850E947B13292F2295B3
:104F40002F70903450F49F70223080F0911599F0BA
:104F5000F8019681903178F489CE2A5F2F70223043
:104F600078F0C8010E944318F72C80CE911519F0F3
:104F7000811509F47BCE805E883008F477CEF1CFBE
:104F8000803F08F473CE815F8330F7CF89E0E3E997
:104F9000F4E0DF011D928A95E9F74DCF981315C013
:104FA00090919304F801808198130FC061100DC097
:104FB000B682C8010E94431889E0F801A3E9B4E071
:104FC00001900D928A95E1F7C2CDC8010E94881325
:104FD000811509F4BEC0611409F4BBC08091990425
:104FE000803208F4ABCD1E821F821886198680910C
:104FF0009304909194049A838983FC82EB8280913C
:1050000097048D83BF82CE0101960E94431896CDEE
:10501000D0909904F0E1DF1638F483E994E00E941F
:10502000431889E0D5019FCE511409F490CD909199
:105030009404F8018181981311C0909193048081A8
:1050400098130CC061100AC0D682C8010E94431890
:1050500089E0D5011D928A95E9F779CDC8010E94B2
:105060008813811509F475C0611409F472C0809128
:105070009904803208F462CD1E821F821886198638
:1050800080919304909194049A838983FC82EB82AB
:10509000809197048D83DF82B6CF0E94B6130E9461
:1050A0004B158816990608F058C0511409F44FCDD5
:1050B000611409F44EC090919404F8018181981311
:1050C00030C090919304808198132BC080919504F7
:1050D00090919604E81AF90A60E083E994E00E944E
:1050E000B6138091C0049091C104E816F90608F047
:1050F00063CF8091990480FD5FCF803108F45CCF4D
:10510000D80116968C931697982F907F903F09F4AC
:1051100050CF982F907F905F8F70892B16968C932D
:1051200048CFC8010E948813811571F0609147042F
:1051300070914804C80170DC811509F4FFCC89E046
:10514000E3E9F4E0DF0186CF8091990481608093E8
:105150009904C8010E944318FACC89E0F501119224
:105160008A95E9F782CDA1E2B0E0E9EBF8E20C9490
:1051700031334C8F5D8F6E8F7F8F082F88A3192F4F
:1051800099A3F82EE92E811509F4A3C040E0692FF8
:105190008C8D9D8D0E949A139C01111549F01092DF
:1051A000C8049093C7048093C604109243040AC0B5
:1051B0008091C6049091C7048217930719F481E087
:1051C0008093C804198E1A8E1B8E86E0FE017C9691
:1051D000DE01539601900D928A95E1F78091C50406
:1051E00082FF21C080919E0490919F04892BD9F069
:1051F0000E9493092091450430914604821B930B31
:1052000020919E0430919F048217930738F080917B
:10521000440482FD03C082E00E9418050E949F0999
:1052200081110E944905F11461F00F8B188F61E024
:10523000CE0143960E94B61361E0CE0143960E94D0
:10524000B6130F8B188F89E0FE017396DE011A9654
:1052500001900D928A95E1F7CE010A9629DC811121
:1052600010C02091490430914A0489E0FE013A9629
:10527000DE01119601900D928A95E1F78E858111DC
:105280002CC019E080914A0490914904891741F09B
:10529000189FC0011124855B9B4F0ADC811144C01B
:1052A0008E85811112C08091140181110EC08C85F0
:1052B0009D852091470430914804821B930B8F3FBA
:1052C0009F4318F081E080931401A196E6E00C94CE
:1052D0004D33911509F476CF68CF822F90E0019677
:1052E000877099273817190671F40E941C0E1092C6
:1052F000490410924A0489E0E3E9F4E0DF011D92D9
:105300008A95E9F7BECF99E0929FD0011124A55B61
:10531000BB4FFE01319601900D929A95E1F7809373
:1053200049040E940E05ADCF80914A0490E0019699
:105330008770992780934A04A5CFA6E0B0E0E3EAFE
:10534000F9E20C9433330E9493098C018091560248
:10535000909157028017910771F019821A820E946A
:105360009309BC0149815A8180E090E0FCDE1093F2
:105370005702009356022696E4E00C944F33A6E0C1
:10538000B0E0E5ECF9E20C9435339093530280934E
:105390005202811520E2920730F40E949F0D26965A
:1053A000E2E00C94513380EF89838A830E94930951
:1053B0008160BC0149815A8181E091E0D4DEEFCF68
:1053C000A6E0B0E0E6EEF9E20C9435339093530298
:1053D00080935202811520E2920730F40E94E60D7C
:1053E0002696E2E00C94513380EF89838A830E94F1
:1053F00093098160BC0149815A8181E090E0B3DE6C
:10540000EFCFCF93DF93D82FC92FB9DF8091BA04A4
:105410009091BB040E94FD0B8D2F9C2FD1DFDF915B
:10542000CF9108950F931F93CF93DF938C01862F15
:1054300063E173E00E943615892B91F4C091130348
:10544000D0911403209761F0F8018281833039F400
:10545000CE01D7DFCE01D5DFCE01D3DF01C0E0F72B
:10546000DF91CF911F910F9108950F931F93CF93C9
:10547000DF938C01EB0163E173E08C2F0E94361502
:10548000892B09F057C0FE01FF27D80112968C9195
:105490001297E75EFD4F8130A9F415968C9182FD3D
:1054A0004EC080FF4CC082E08083809115039091B4
:1054B00016030097B9F48091130390911403009799
:1054C000C9F110C08230A1F515968C9182FD26C0DD
:1054D00080FD0AC083E080838091170390911803B8
:1054E0000097F1F04CDF26C084E08083809119039F
:1054F00090911A030097B1F78091130390911403D0
:10550000009701F17EDF80911503909116030097BB
:1055100049F78091130390911403E4CF85E08083D1
:105520008091130390911403009721F06ADFF1CF6B
:1055300086E08083DF91CF911F910F91089581E0E4
:105540008083B9CF8091150390911603B8CF0F9344
:105550001F93CF93DF938C01EB0163E173E08C2FFA
:105560000E943615892BA1F48091BA049091BB0456
:105570000E94FD0BDD27C75EDD4F8881F801128296
:1055800018828330E9F048F4813059F0823081F09C
:10559000DF91CF911F910F9108958430B1F0853044
:1055A000B9F78091130390911403009789F306C013
:1055B0008091150390911603009799F301DFE8CFCE
:1055C0008091170390911803F7CF80911903909160
:1055D0001A03009799F720911303309114038091D7
:1055E00015039091160321153105F9F2009731F753
:1055F000C901E4CFCDB7DEB7AC970FB6F894DEBFE4
:105600000FBECDBF85B7806885BF85B7806885BF71
:1056100084B7877F84BF0FB6F894A8958091600007
:10562000886180936000109260000FBE80E890E077
:105630000FB6F89480936100909361000FBE81E0F3
:105640008093110183E497E09093AF018093AE01C2
:105650000E946B070E9477140E94F6140E94AE12FB
:105660000E94270B0E94840B8091E200846080934B
:10567000E200789480915102811599F08091E900BF
:105680001091EC008F70179511271795182B109219
:10569000E9008091E80083FD0E94880E1F7010933E
:1056A000E90082E084BD93E095BD9AEF97BD8093B9
:1056B0006E000E94D113811102C00E9475170DE285
:1056C00011E0D8018D918D018F3F11F00E944507A7
:1056D000B1E002331B07A9F702E311E0A1E4EA2ECF
:1056E000A1E0FA2EF80181918F018F3F11F00E9405
:1056F0004507E016F106B1F78AE0E5E4F2E0DF01E4
:10570000282F1D922A95E9F7E1E2F2E0DF011D92D0
:105710008A95E9F780E090E00E949A33833E9E4F9D
:1057200021F40E94D113811129C063EE7EEF80E045
:1057300090E00E94C83360E082E090E00E94AE33C7
:1057400081E080933E0461E083E090E00E94AE330C
:1057500060E074E184E090E00E94C8330E94751715
:1057600040E050E0BA018FE090E00E94C03340E09A
:1057700050E0BA0183E190E00E94C03382E090E003
:10578000D1D780932D0284E090E0D4D79093C504C4
:105790008093C4040E948B16EFEFF6E721E0E150FE
:1057A000F0402040E1F700C000000E948B1680917D
:1057B000450280FF07C06FEF7FEF80E090E0E8D701
:1057C0000E940B0C83E090E0ADD70E94F60380E0CE
:1057D00091E0909379028093780280915102853014
:1057E00049F480915102853009F45CC00E941C0E7E
:1057F0000E94D1080E948B16FEE2AF2EF2E0BF2E6F
:1058000005E412E0D801F501219131918D919D912E
:1058100048E352E04E175F0709F47AC028173907AA
:1058200099F3E5E48E2EE2E09E2E512CD401ED900A
:10583000FD904D01F501619071905F016E147F0440
:1058400051F16E247F24412CCC24C394D12CC3016C
:105850008C219D21892BB1F049825A820E949309A3
:105860009C838B83F1E0FD8391E097012C213D2106
:10587000232B09F490E09E8349815A816B817C81BE
:105880008D8171DC4394CC0CDD1C2FE04212DFCF04
:10589000F501F292E292539435E05312C7CF0E9481
:1058A000300A3BC080915102843021F110922B02CA
:1058B00048E150E080E40FB6F894A895409360006A
:1058C0000FBE8093600083B7817F846083BF83B7FE
:1058D000816083BF7894889583B78E7F83BF0FB62E
:1058E000F894A89580916000886180936000109280
:1058F00060000FBE0E948B16E5E4F2E08191919169
:10590000892B09F0BCC492E0EF34F907B9F769CFED
:105910002817390709F085CF10DDE0909E03F0903D
:105920009F03E114F10491F180903C0290903D02BC
:10593000A0903E02B0903F020E94300A6819790997
:105940008A099B098090380290903902A0903A020F
:10595000B0903B02681579058A059B05B8F0C70130
:105960000E949F0D10929F0310929E0310923C0282
:1059700010923D0210923E0210923F0210923802A5
:105980001092390210923A0210923B02C090260403
:10599000D0902704C114D10439F1A0902804B0900C
:1059A00029040E9493097C01EA18FB08C6010E94A1
:1059B0004B158E159F05C0F42091260430912704C5
:1059C000C9019927287F3327232B09F080C054E091
:1059D000880F991F5A95E1F78A559C4FDC0115965F
:1059E0002C9122FF0E9410128091B70480FF1CC0EE
:1059F0008091130182FF18C00E949309BC0180911D
:105A00002A0490912B049B01281B390B80910C01D7
:105A100090910D012817390738F041E080912C044E
:105A200090912D040E946C1180911D03811569F0E5
:105A30000E94930920911E0330911F03821B930B38
:105A40008F3F9F4710F40E943A0D0E94D108909119
:105A50004002891721F0809340020E94300A809111
:105A60005102843009F0B9CE83E08093E90080913F
:105A7000E80082FFB2CE8091E80090E085FF05C08B
:105A80000E94F60A811531F191E08091E8008B7750
:105A90008093E800911509F4A0CEE0905402F090B4
:105AA0005502E981E114F10499F1EE3F09F051C08A
:105AB0008A81833020F08550833008F04AC0EA8123
:105AC000EE3008F046C0F0E0EA50FC4CA1C580E0A2
:105AD00090E084CF40E2C42ED12CFE0131967F01AC
:105AE0008091E80085FD0AC08091E8008B77809363
:105AF000E8000E94F60A811599F3C6CF8091F10063
:105B0000D7018D937D01B1E0CB1AD10849F7BCCF05
:105B1000E43148F4E11549F0E150E33130F4F0E0CC
:105B2000EC5FFB4C75C5EE3F51F28FEFD4C31A8288
:105B300089E08B830EC08A81823081F08330B1F09E
:105B4000813099F70E94300A79D56B837C838D83ED
:105B50009E83CE0101960E94460B3FCE88E290E0E4
:105B6000E1D51B821C821D828E83F3CF80914F0270
:105B700090915002892B69F3FE013196D8018C91E6
:105B800011969C910E5F1F4F928383833296B2E0F1
:105B90000F341B0799F7DDCF8A81823031F66B8194
:105BA0007C818D819E814AD588E290E0D7D5D1CF86
:105BB0004C816B818A810E94071398278927982737
:105BC0009E838D83C6CF2D813E81322723273227A6
:105BD0004C816B818A810E94A70CBBCF0E94EA1383
:105BE000B8CF80E18A83B5CF1A8287E8A2CF8C81B3
:105BF0008D3108F0AECF8A809B8098248924982428
:105C0000A12CB12C8E010F5F1F4F7801E80EF11C03
:105C1000E016F10609F49DCF80E0E7E88E169104C6
:105C2000A104B10420F4C40187589C4F7BD5D8014E
:105C300014968C930F5F1F4FBFEF8B1A9B0AAB0A12
:105C4000BB0AE6CF80914F0290915002892B09F454
:105C500080CF8C818D3108F07CCF882E912CA12CA7
:105C6000B12CCA80DB80DC24CD24DC24E12CF12C97
:105C70008E010F5F1F4F412C512C320148145904E3
:105C80006A047B0408F065CFE7E8CE16D104E1048E
:105C9000F10438F4D80114966C91C60187589C4FD2
:105CA0005DD5BFEF4B1A5B0A6B0A7B0AEFEFCE1A8A
:105CB000DE0AEE0AFE0A0F5F1F4FE0CF0E943B177D
:105CC00048CF84E08FCF8C818D3108F042CF882E71
:105CD000912CA12CB12CCA80DB80DC24CD24DC24C7
:105CE000E12CF12C412C512C32018E010B5F1F4F06
:105CF000481459046A047B0408F02BCF80E0F8E5CF
:105D0000CF16F2E0DF06E104F10418F4C60189962B
:105D100009D5D8018D938D01BFEF4B1A5B0A6B0A31
:105D20007B0AEFEFCE1ADE0AEE0AFE0AE1CF2C81E3
:105D3000022F10E02D3108F00CCF8A819B8198272B
:105D4000892798272C01612C712C8835F2E09F0758
:105D500008F0FFCE822E912CA12CB12C48E552E008
:105D600060E070E04419550966097709421751054A
:105D70006105710508F4EDCE20914F02309150027B
:105D8000232B09F03EC01C0129E2220E311C80FBAE
:105D9000EE24FF24E0F880FF0BC08896C3D49D81D9
:105DA00089279827892781159C4711F48FEF8D83C8
:105DB000D501C401840D951DA61DB71D80FF19C016
:105DC000680141E0C41AD108CE0105968C0D9D1DD5
:105DD0009CA78BA7C101800F911FA4D4ABA5BCA524
:105DE0009C9181159C4721F48FEFEBA5FCA5808346
:105DF0008601FE013196EE0DFF1D2FEFE016F10634
:105E000038F08E010F5F1F4FC12CD12C760125C0B9
:105E10009481858181159C4711F42483258342E078
:105E2000E40EF11C3296EACF58E5451652E05506CD
:105E30006104710430F4D80114966C91C201899602
:105E40008DD4BFEFCB1ADB0AEB0AFB0AEFEF4E1A39
:105E50005E0A6E0A7E0A0F5F1F4FC814D904EA0457
:105E6000FB0410F376CE80914F0290915002892B63
:105E700009F46FCECE0101960E94460BFFEF21EE92
:105E800034E0F15020403040E1F700C0000098CCF1
:105E900088E0E5E1F1E0DE01919601900D928A95AE
:105EA000E1F7FE0132968FE1DF011D928A95E9F755
:105EB00086E0898388E07F96DE01159601900D9239
:105EC0008A95E1F746CE80E5898381E08A831B824B
:105ED0001C823FCE8B819C81092E000CAA0BBB0B30
:105EE00035E0880F991FAA1FBB1F3A95D1F7AC0167
:105EF000BD01405E5F4F6F4F7F4F481759076A07DC
:105F00007B0708F426CE8035E1E09E07A105B105A8
:105F100008F01FCE4135F1E05F076105710520F003
:105F200040E551E060E070E0481B590BBC01645251
:105F30007B4FCE010196C0D30CCE4AE150E06FEF0B
:105F400070E0CE010796D7D380914F028983EA8211
:105F50001B821C8284E08D838EE006CE81E090E07F
:105F6000909355028093540282E390E09093440210
:105F7000809343020E9493099093420280934102CE
:105F8000E8CDE114F10481F1D0904502C0904E02B9
:105F900000914102109142020E949309801B910BD3
:105FA0008536910540F1C6FE26C0D0FE24C00E9471
:105FB0009309909342028093410280914302909111
:105FC000440201979093440280934302892B61F429
:105FD000109255021092540281E090E0909350028A
:105FE00080934F02E12CF12C80914F028983EA8249
:105FF000809143029ECD82E390E09093440280938F
:106000004302F2CF1092500210924F02A2CD0B81A8
:106010001C8140E250E06FEF70E0CE0101966BD33F
:1060200020E134E042E050E080E090E0F901659149
:1060300075910617170740F4DE0111968A0F9B1F12
:10604000FC0171836083CA01F4E0203D3F0709F43D
:1060500080CDAC014E5F5F4F245F3F4F4132510511
:1060600028F377CD2B813C8180E194E0FC014591C0
:1060700055914217530709F41FC10C9644E08C3D1B
:106080009407A1F752CD8B819C8100E114E0F801C7
:10609000259135918217930709F41FC1045F1F4FA3
:1060A000F4E00C3D1F0799F7EE24EA94FE2C30C172
:1060B0000E94D4124ECDEB81E93008F04ACDF0E0D9
:1060C000E95EFB4CA5C2FE0132968EE1DF011D9216
:1060D0008A95E9F788E089838B838C8383E088A3A2
:1060E00038CD8C819AE0F92E8E010F5D1F4FF8019B
:1060F0002F2D11922A95E9F7B8010E943615898350
:10610000F801DE01129601900D92FA94E1F721CD8B
:106110001C818AE0FE013596DE01919601900D9278
:106120008A95E1F789A19AA10E945E079AA389A3A3
:106130008BA19CA10E945E079CA38BA38DA19EA115
:106140000E945E079EA38DA38FA198A50E945E0763
:1061500098A78FA38FEF183060F43AE0139FB00137
:10616000112467557D4F4AE050E0CE01819614D34B
:1061700080E089830E946B07ECCC2C816AE0CE0121
:106180008196DC01E62F1D92EA95E9F7283080F42C
:10619000629FB001112467507D4F4AE050E0B2D2B7
:1061A00080E089838AE0FE01B196DE01129686CEF8
:1061B0008FEFF7CF1C818AE0FE013596DE019196C4
:1061C00001900D928A95E1F78BA19CA10E945E0738
:1061D0009CA38BA38FEF183060F4FAE01F9FB001EF
:1061E000112467507D4F4AE050E0CE018196D4D211
:1061F00080E089830E947714ACCC2C8166E0CE01CC
:106200008196DC01E62F1D92EA95E9F7283060F4CB
:10621000629FB0011124675B7C4F46E050E072D270
:1062200080E0898386E0BFCF8FEFFBCF1C8186E0C3
:10623000FE013596DE01919601900D928A95E1F767
:1062400089A19AA10E945E079AA389A38BA19CA110
:106250000E945E079CA38BA38FEF183060F4F6E0DA
:106260001F9FB0011124675B7C4F46E050E0CE01D8
:10627000819692D280E089830E94F6146ACC809144
:106280002C02811509F4ADCAA0E1A9BDB2E1B9BDE6
:1062900009B400FEFDCF8091D8008F7D8093D80097
:1062A0008091E00082608093E0008091E00081FDB9
:1062B000FCCF0E941C0E95CAFC01369625913591A3
:1062C0002115310509F431CC4FE150E0BE016E5F7C
:1062D0007F4FF901099589833CCCF80138962591C7
:1062E00035912115310509F4DFCE4CE150E0BE01B6
:1062F0006B5F7F4FC801F90109957C01892B41F43F
:10630000F8013A9685919591009711F0FC01099555
:10631000E9821FCC1F921FB61F9211248F939F9367
:10632000AF93BF9380912B02811113C08091F00134
:106330009091F101A091F201B091F3014196A11D5C
:10634000B11D8093F0019093F101A093F201B093FD
:10635000F301BF91AF919F918F911F901FBE1F902E
:10636000189578941F921FB61F9211248F939F93B4
:10637000AF93BF938091F0019091F101A091F20150
:10638000B091F3010196A11DB11D8093F00190938E
:10639000F101A093F201B093F301BF91AF919F91EE
:1063A0008F911F901FBE1F9018951F920F920FB6CE
:1063B0000F9211242F933F934F935F936F937F938B
:1063C0008F939F93AF93BF93EF93FF938091E100DF
:1063D00082FF09C08091E20082FF05C08091E10048
:1063E0008B7F8093E1008091DA0080FF24C0809150
:1063F000D80080FF20C08091DA008E7F8093DA0081
:106400008091D90080FFA9C080E189BD82E189BD6A
:1064100009B400FEFDCF81E0809351028091DF013D
:10642000811109C00E94270B0E94840B8091E20019
:1064300084608093E2008091E10080FF1AC0809127
:10644000E20080FF16C08091E2008E7F8093E20020
:106450008091E20080618093E2008091D8008062A8
:106460008093D80019BC85E08093510283E080932B
:1064700011018091E10084FF2FC08091E20084FF30
:106480002BC080E189BD82E189BD09B400FEFDCF4A
:106490008091D8008F7D8093D8008091E1008F7E1D
:1064A0008093E1008091E2008F7E8093E2008091F2
:1064B000E20081608093E2008091DE01811509F4A1
:1064C00052C084E08093510280915102843009F0DF
:1064D00052C082E0809311018091E10083FF2CC0C3
:1064E0008091E20083FF28C08091E100877F809344
:1064F000E10082E0809351021092DE018091E10080
:106500008E7F8093E1008091E2008E7F8093E20095
:106510008091E20080618093E20042E060E080E0F0
:106520000E94540B8091F00088608093F00081E01D
:106530008093110180931001FF91EF91BF91AF9172
:106540009F918F917F916F915F914F913F912F918B
:106550000F900FBE0F901F90189519BC109251020A
:106560001092DF0168CF8091E30087FF02C083E0D3
:10657000A9CF81E0A7CF81E0ADCF1F920F920FB6D8
:106580000F921124EF92FF920F931F932F933F933B
:106590004F935F936F937F938F939F93AF93BF932B
:1065A000CF93EF93FF9309EE10E0F8018081C09143
:1065B000EC008F70C795CC27C795C82B108280EF51
:1065C000E82EF12CF7018081877F808378940E94E8
:1065D000880EF8011082F701808188608083CF7077
:1065E000F801C083FF91EF91CF91BF91AF919F913F
:1065F0008F917F916F915F914F913F912F911F915B
:106600000F91FF90EF900F900FBE0F901F90189575
:10661000EE0FFF1F0590F491E02D0994082E817074
:1066200006940694811D0694811D0694811D06948E
:10663000811D0694811D0694801D08956927962763
:10664000692778278727782708952F923F924F92BE
:106650005F926F927F928F929F92AF92BF92CF92F2
:10666000DF92EF92FF920F931F93CF93DF93CDB7FB
:10667000DEB7CA1BDB0B0FB6F894DEBF0FBECDBF73
:1066800009942A88398848885F846E847D848C8444
:106690009B84AA84B984C884DF80EE80FD800C814D
:1066A0001B81AA81B981CE0FD11D0FB6F894DEBF30
:1066B0000FBECDBFED010895FB01DC0102C00590C6
:1066C0000D9241505040D8F70895FB01DC0104C001
:1066D0008D910190801921F441505040C8F7881BDA
:1066E000990B0895FB01DC0102C001900D9241500D
:1066F0005040D8F70895DC0101C06D9341505040DF
:10670000E0F70895DC01CB01FC01F999FECF06C04A
:10671000F2BDE1BDF89A319600B40D92415050405F
:10672000B8F70895F999FECF92BD81BDF89A9927DF
:1067300080B50895A8E1B0E042E050E0E5CFDC018B
:10674000A40FB51F4150504040F0CB01840F951F5E
:106750002E9105D041505040D8F70895262FF99931
:10676000FECF92BD81BDF89A019700B4021639F0B0
:106770001FBA20BD0FB6F894FA9AF99A0FBE089581
:106780000396272FECDFEADF252FE9DF242FE7CF61
:106790000196272FE4DFE2CFDC01CB0102C02D916F
:1067A00005D041505040D8F70895262FF999FECFD3
:1067B0001FBA92BD81BD20BD0FB6F894FA9AF99A1E
:1067C0000FBE01960895F894FFCF650F8B0F910FC0
:1067D0008B0F910FE30F0410910F0A11171158201E
:1067E0005E204A20522064206A207020482F632FA8
:1067F0006A2FA92DA92D9D2FAE2FC12F0230073052
:106800003230433058305B30972D9B2DCC2DD82D16
:10681000E32DEE2D952D952D952D952D332FF12DC5
:10682000F42DF72D222E5E2E612E632E972E6330CF
:1068300071308830A92DA92DBD30DA30FD301631E8
:106840009009710C870C7D0A8C0C680CAF0000005D
:106850000100010101888EA1C2C87EACEC00442277
:106860006D3B011901AC0041025A027A029190F786
:10687000F5F637F0F1F467663635349796949593CC
:1068800092E200E900EA00B500B600B700CD00834F
:1068900001CC008A019201940121022302240225E5
:1068A00002260227022A02B300B4006F0070009F84
:1068B00001CB019F02A002E200E900EA00B500B6A8
:1068C00000B700CD008301CC008A01920194012120
:1068D00002230224022502260227022A02B300B460
:0E68E000006F0070009F01CB019F02A002001C
:00000001FF
